:040000006F00204429
:100004000000000000000000480200004A02000056
:100014000000000040040000000000000000000098
:100024004004000040040000000000000000000044
:10003400401A00000000000040040000000000001E
:10004400400400004004000040040000400400009C
:10005400400400004004000040040000400400008C
:100064003815000040040000400400004004000073
:10007400400400004004000040040000400400006C
:10008400400400004004000040040000400400005C
:10009400400400004004000040040000400400004C
:1000A400400400004E1A0000400400004004000018
:1000B400161A000066190000400400004004000005
:1000C400400400004004000040040000400400001C
:1000D4004004000040040000400400005A180000DE
:1000E40040040000400400004004000040040000FC
:1000F40040040000A0180000400400004004000078
:1001040040040000400400004004000040040000DB
:100114004004000000000000000000000000000097
:1001240000000000000000000000000000000000CB
:0C013400000000000000000000000000BF
:10014000397101436EC619A0397141536AC866CA34
:1001500062CC5ECE19A0397101535AD056D252D416
:100160004ED64AD826DA22DC06DE3301614082828E
:1001700041114AC026C222C406C68282B24D410144
:10018000024D924C224CB24B4101024B924A224A00
:10019000B2494101024992442244B2404101828065
:1001A0003D432A876373C3029377F700BDEFADE544
:1001B000937606FF3D8ABA960CC34CC30CC74CC756
:1001C0004107E36BD7FE11E28280B306C3408A0683
:1001D0009702000096966780A6002307B700A30643
:1001E000B7002306B700A305B7002305B700A30493
:1001F000B7002304B700A303B7002303B700A3028B
:10020000B7002302B700A301B7002301B700A30082
:10021000B7002300B700828093F5F50F9396850011
:10022000D58D93960501D58D61B7939627009702DA
:10023000000096968682E78086FA9680C1171D8F09
:100240003E96E374C3F8A5B701A001A0EFF25FF2F8
:100250000545EF00D0289922EF10101571651305A0
:100260000520EF10D019B707002083A507163785A2
:10027000000013054592EF50107B0925AA853785AC
:10028000000013054593EF50107AEF30605EEF30B9
:10029000E055014501B7EFF2BFED371402401C40B5
:1002A0003707FF08411193E717001CC05C40F98F26
:1002B0005CC01C403707F7FE6D17F98F1CC01C404F
:1002C0003707FCFF7D17F98F1CC05C40370701FF23
:1002D0007D17F98F5CC0B7079F001CC4EF00300783
:1002E00002C402C6B7270240054798C31C404167B5
:1002F000B7160240D98F1CC03706020005679C4222
:10030000F18F3EC6A24785073EC4B24781E7A247A8
:10031000E397E7FEB71702409C431397E700635744
:10032000070685473EC6324785476313F706B7176A
:100330000240D843B706C1FFFD16D8C3D843D8C37F
:10034000D84313670740D8C3D843758FD8C3D84361
:10035000B7061100558FD8C39843B7060001558FD3
:1003600098C3984393166700E3DD06FED843B7169B
:100370000240719BD8C3D84313672700D8C32147D5
:10038000DC42B18BE39EE7FE410129B502C661BFA5
:10039000372702401C43F19B1CC3FDB7B716024030
:1003A000DC42370700201146B18B13070716638F15
:1003B000C70221466381C70495EB9C42918B9DC780
:1003C000B7470F00938707241CC3B7170240DC43CD
:1003D000918393F6F700B707002093870700B6973D
:1003E00094231C43B3D7D7001CC38280B7177A006D
:1003F00093870720D1BFDC42D4424166C983BD8BBD
:10040000F18E890745466393C700C94781EEB74619
:10041000024083A60680C18A89CEB7167A009386E9
:10042000062021A8B7160240D4421396E600E356F0
:1004300006FEB7163D0093860690B387D70269B7CC
:1004400001A0970100209381E15117510020130171
:1004500061BB178500001305A5ED97050020938566
:1004600065BA1386018263FAC5008322050023A0C2
:10047000550011059105E3EAC5FE138501829385B8
:1004800081B76377B500232005001105E36DB5FE44
:10049000FD42739002BC8D427390428093028008AB
:1004A0007390023097020000938202B693E232000A
:1004B00073905230EFF03FDE97020000938242D9F2
:1004C0007390123473002030B727014093870740A0
:1004D000631FF500EFF2DFC9854513050020EF002B
:1004E0001018814513050020EF00701765B1828058
:1004F0005C413707F1E01307F7EF944D7D8F9C4186
:10050000D58FD44DD58FD441A206D58FD98F5CC15C
:100510001C4537F7F1FF1307D77FD4457D8F9C49E2
:10052000D58F94458606D58FD98F1CC55C55370766
:1005300010FF7D177D8FDC29FD1793F7F70FD2078A
:10054000D98F5CD582801C4589C593E717001CC5EF
:100550008280F99BEDBF1C4593E787001CC5828014
:1005600008450D81058982801C4593E747001CC51D
:10057000828008450981058982801C4591C537071D
:100580005000D98F1CC582803707B0FF7D17F98FC7
:10059000D5BFA54763F7B7048D47138765FF3307BA
:1005A000F7020328C5009D47B397E70093C7F7FFFD
:1005B000B3F70701B396E600DD8E54C5994763E3B0
:1005C000C70495477D163306F6025859FD47B39781
:1005D000C70093C7F7FFF98F3396C5005D8E50D9DA
:1005E00082800D473387E502032805019D47B397B5
:1005F000E70093C7F7FFB3F70701B396E600DD8E78
:1006000014C96DBFB14763E2C7029547651633064B
:10061000F6021859FD47B397C70093C7F7FFF98F44
:100620003396C5005D8E10D9828095474D163306EE
:10063000F6025855FD47B397C70093C7F7FFF98FE8
:10064000B395C500DD8D4CD582806845420541815A
:10065000828008416D8D3335A00082805C4191C558
:1006600037070004D98F5CC18280370700FC7D17F3
:10067000F98FD5BF3C4989C593E707083CC98280FB
:1006800093F7F7F7E5BF3C4989C593E707043CC9F1
:10069000828093F7F7FBE5BF3C4993F7F7FD3CC930
:1006A0003C49DD8D2CC98280EFF29FACB7066745CF
:1006B000B7270240938636123797EFCDD4C313077E
:1006C000B79AD8C3D4D3011198C7D45B1387470313
:1006D00013962600E34B06FED45737250140130539
:1006E000054093E60620D4D7DC5BB7060020D58F03
:1006F0001CC31C431C4537070E00D98F1CC51C4565
:1007000093E717001CC53C4993E707043CC91C4507
:1007100093E787001CC52A842285993575FD372506
:100720000140832785401305054093E747001CC51A
:100730002A8422853D3D75FD372501400546C94582
:10074000814613050540B1352546230401003727AE
:100750000140B70550001C84637FF60423040100A8
:10076000A54621461C8463FFF606231501002304D9
:10077000010095461C8463F1F60E38853C85994648
:100780000D46B3F7D7020565130505803357D70229
:10079000B3D7C702BA97C207C1837C85B727014088
:1007A00003A78740799B23A4E7403C8505611D8D05
:1007B00042054185C5B283278740CD8F2324F7406A
:1007C00083270740898BEDDF1C848326C7440810EC
:1007D0008607AA972396D7FE1C84850793F7F70F01
:1007E0005C8495BFA30401009C846378F6001C849C
:1007F000850793F7F70F5C84B5B798849C840C1039
:100800000607850786072E97AE970357C7FE83D73F
:10081000C7FE63FDE7029C848607AE9783D7C7FEB9
:100820007C859C84988485078607AE9783D5C7FE10
:10083000931717001810BA972396B7FE9C84388533
:100840000C1085078607AE972396E7FE9C848507E4
:1008500093F7F70FDC8449BF1C8410103885890793
:100860008607B29783D7C7FEBA97C207C1837C8534
:100870001C84850793F7F70F5C84EDBD03A54182C7
:1008800082805841032805004C45370601409307F4
:1008900006403E979346F8FFB1C583250640F58D87
:1008A0002320B640D043F18ED4C31443B3E60601EF
:1008B00014C3184190479346F7FF758E90C7D047F1
:1008C000F18ED4C7144541466399C6009447D98E2A
:1008D00094C7D447558FD8C78280B6979443558F15
:1008E00098C382801C43F58F1CC38280B7070140E8
:1008F0001387074083A70740584B698F09C77D8D31
:100900003335A000828001458280B707014023AAC9
:10091000A74082809C4513F7070113F8F70001C731
:10092000D8413368E8008E2113F7F50F39C3184119
:100930008146854E3D4F930F800293028004214EE5
:100940003396DE00B3F8C5006311160393982600B2
:1009500033131F011343F3FF3377E300B318180178
:1009600033E7E800639FF70550C98506E39AC6FDA3
:1009700018C11307F00F6375B70454412146854E23
:100980003D4F930F800293028004414EB398CE00F6
:1009900033F715016392E80213172600011733138A
:1009A000EF001343F3FFB376D3003317E800D98E7B
:1009B000639DF701232A15010506E319C6FD54C1FD
:1009C0008280E39457FA10C94DB7E39757FE232866
:1009D0001501DDB708456D8D3335A000828048458F
:1009E0006D8D3335A00082800CC9828019C20CC97C
:1009F00082804CC98280370700C0B377E5006395D9
:100A0000E708370701405C439356B501584F9D8A6C
:100A10009DE6F99BB70600FFFD16758F89C99316F1
:100A20000501C182D58FB706FF01758D498FB706C5
:100A30000007D58FB7060140DCC2D8CE82800546BC
:100A40006396C600F59BB70680FFF9B70946639623
:100A5000C600ED9BB706E8FFC1B70D466396C6001A
:100A6000DD9BB706FCFF4DBF11466397C60093F7A9
:100A7000F7F3B706C0FF4DB71546E391C6FA93F7F3
:100A8000F7CFB706E0FF49BF370700406391E702A1
:100A9000B7070140D84F4205B367A70089E5134562
:100AA000F5FFB377E500370701405CCF8280A9E30B
:100AB00037080140B7073000032648001317050127
:100AC000B376F50041836396F602B70600F9FD168A
:100AD000B377D60003264800F18E2322D80091C5B3
:100AE000558112053315A700C98F370701405CC334
:100AF00082809317B50063D007029357050193F6E0
:100B0000F7008D47B397D70093C7F7FFF18FB7066C
:100B10000007D58FE9B7935755019207B317F70030
:100B2000E5B713F7C50F93F73500B7050140BA9540
:100B300094458A073D473317F7001347F7FF758F32
:100B400098C598453315F500598D88C58280EFF218
:100B50002FE237F4FF1F032744723706003E41118E
:100B6000931797019346F7FFF18F060737063E006C
:100B7000718FD98F3706000113979600718FD98F27
:100B8000BD824167F98ED58F02C202C402C623A47A
:100B9000F1820357847285452390E1820327047212
:100BA0001305D00323A6E1820327447023A2E18228
:100BB0008D2C8327447037073A101307077093F77B
:100BC000F7F06380E7106361F7023707321013070D
:100BD00007706380E70637073710130707706387CE
:100BE000E70841016FF00FDB37073B101307077071
:100BF000638BE70A37073D1013070770E393E7FE9F
:100C000085452165CD3BB7140140E177130480048D
:100C10004C00138504807C8222C6ED39856793875A
:100C2000C7334C00138504C07C8222C6E531F977B6
:100C30000DA085452165C133B7140140930700E03D
:100C4000130480044C00138504C07C8222C6D93171
:100C500089674C00371501407C8222C665398D4773
:100C60007C8222C64C001385044025A8B71401409D
:100C7000E17793870770130480044C001385048088
:100C80007C8222C641399307D0E34C00138504C00F
:100C90007C8222C64131F9777C8222C64C0037150E
:100CA00001408D393DBFB7140140E1771304800442
:100CB0004C00138504807C8222C6A939930740200A
:100CC0008DB7B7140140E177130480044C001385FD
:100CD00004807C8222C63D398967F51799B723A81D
:100CE000A182828003A70183854714216310F70244
:100CF0001C31639CE7023C21960793E707F837E72E
:100D000000E093F7F70F36972300F740054793D796
:100D100056003317D700544189CE938707048A07BA
:100D2000B7E600E0B69798C38280EDF33C219607C2
:100D3000F9B793870706E5B7B7160240DC42374795
:100D4000FF7F7D17F98F5D8DC8C282803717024003
:100D50005C439146B18B638CD706A146638ED70660
:100D6000BDE71C43918BA5C7B7470F0093870724A6
:100D70001CC1371602405C423707002013070701E9
:100D80009183BD8BBA9794231C41B3D7D7005CC124
:100D90005442A1829D8ABA969422B3D6D70014C534
:100DA0005442AD829D8A36971423B3D6D70054C5DA
:100DB0005842634C07005C42B98313F737009387AE
:100DC0004180BA979C23B3D7F6021CC98280B7171B
:100DD0007A009387072069BF5C435843C166C98383
:100DE000BD8B758F8907C5466393D700C94701EF4F
:100DF0003747024003270780418B09CF37177A0016
:100E00001307072021A83717024058439316E7001D
:100E1000E3D606FE37173D0013070790B387E702B6
:100E200081BF99C5371702401C4F5D8D08CF828066
:100E3000B7170240984F1345F5FF798D88CF828010
:100E400099C5371702405C4F5D8D48CF8280B71738
:100E50000240D84F1345F5FF798DC8CF828099C5E0
:100E6000371702405C475D8D48C78280B717024044
:100E7000D8471345F5FF798DC8C782801A218D6741
:100E800093870704B6217D8F9E21D58FD621D58FDC
:100E9000F621D58F9625D58FB625D58FD625D58F1A
:100EA000F625D58FD98F1EA19E291EA982801E21CD
:100EB00089C593E707041EA18280C207C18393F707
:100EC000F7FBC207C183C5BF4EA582804A25828039
:100ED0000A256D8D3335A00082801E2137370140F1
:100EE000130707C0C207C1836300E502370700404C
:100EF000630CE500130707406308E500371700405F
:100F0000130707806316E500FA2193F7F7F8D98FE6
:100F10009A2593F7F7CFC207C183D98F37170040BF
:100F20001EA1130707809C416310E5025CD5DE21FA
:100F30001EB5B7370140938707C06314F500BC2581
:100F40001EB985475EA98280C207C1835EB5C5B759
:100F50001A31FD77FD17F98F1EB10358050256218E
:100F60005E2D6577D2211307F7CF7D8FF9772206A3
:100F7000FD17518FB3F70701F22103D8A500C20670
:100F80004207336606013206D18F37360140C20769
:100F9000130606C0C1824183C183631AC5007176FE
:100FA0007D16F18EF2251A06D18EC206C18256A197
:100FB000B71600405AAD9386068098416315D50058
:100FC00038C11EB1828042074183DDBF1E2189C521
:100FD00093E717001EA18280C207C183F99BC20755
:100FE000C183CDBF8357450491C52167D98F231293
:100FF000F5048280C607C583DDBF5E2501C6DD8D91
:101000004EA5828093C5F5FFFD8DDDBF1E2189C5EC
:1010100093E707081EA18280C207C18393F7F7F701
:10102000C207C183C5BF5A2DFD779387F77FF98F1C
:10103000A205CD8FC207C1835EAD8280B717004085
:10104000938707806314F5002CC18280C205C1819B
:10105000E5BFB7170040938707806314F500485138
:1010600082804A314205418182801E294A25ED8FC6
:101070004205418189C76D8D3335A00082800145CD
:10108000828093C5F5FFC205C1810EA98280EFF26F
:101090002F8E1629F577FD17F58FF621DA25797150
:1010A000D58F1EA95625FD779387379FF58FD621BB
:1010B0002A842EC6D58F9625D58FB625D58F5EA5C9
:1010C0005E29C207C18393F7F7CFD98F5EA968085D
:1010D000B539B747014093870780B245631AF404D6
:1010E000A25756246547B387E702C206C1869841D6
:1010F00063D20604060752244206B3D7E702130759
:1011000040064186B3D6E702B3F7E702920663557D
:1011100006028E0793872703B3D7E70213F77700FA
:10112000B367D700C207C1831EA445616FF08F86E5
:10113000925745BF0A07C1B7920793872703B3D7D2
:10114000E702BD8BD58FF9BF91C55E250967D98FA1
:101150005EA582805A25F977FD17F98FD5BF13F761
:10116000F50F85471583B395B7006319F70093070B
:10117000C500984301CED98D8CC3828089469307E0
:101180004501E318D7FE93070501E5B793C5F5FFC1
:10119000F98DDDB793F5F51F4EA182804A211375B5
:1011A000F51F82800A216D8D3335A000828013F7F0
:1011B000F50F85461583B397B6006311D7025A25FC
:1011C000F98F1A2101454207418381CB0545A18151
:1011D000B315B5006D8F3335E00082808946631406
:1011E000D7001A29F1BF5A29E1BFEFE27FF87971E0
:1011F0001306000281450808EFE09FFA8545114576
:1012000002C202C402C631398545130500201139D6
:1012100001451D36371501409307E00F4C001305BB
:101220000580372401407C8202C6EFF0AFEE130543
:101230000440EFF06FA913050440EFF0EFC6AA8554
:10124000239AA1823785000013054594EF40B07DB5
:10125000B7070E003ECE0C08854713050440230255
:10126000F10202C802CA02CC02D0EFF06FA8854595
:1012700013050440EFF02FAD854513050440EFF052
:101280008FC0814513050440EFF04FBD13050440A6
:10129000EFF06FAC930404402685EFF06FAC6DFD6A
:1012A0001305044037240140EFF00FAC93040440D1
:1012B0002685EFF00FAC6DFD37050080B53C1305BA
:1012C00004408545EFF00FBB930500021305044071
:1012D000EFF08FBC45616FE0FFEBEFE27FE90111BA
:1012E000854521453D3E85451165993E37140140B0
:1012F00085678D447C808A85C147130504C03EC440
:1013000026C2EFF02FE1130504C08565EFF0CFEDA5
:10131000896761498A85130504C07C804AC426C256
:10132000EFF04FDF91677C808A859147130504C0F9
:101330003EC4EFF02FDEE1778A85130504C07C8080
:101340004AC426C2EFF00FDDB70704013EC6B70757
:1013500002003EC8B70700028507374400403ECA76
:10136000A1473ECC6C009D4713050480FC863936AE
:10137000854513050480253E05616FE0BFE1EFE27E
:101380009FDDB74400402A891304900C93890480A0
:1013900089454E85353E0DC5CA8513850480B74401
:1013A00000401D361304900C1389048085454A853E
:1013B000053611CD13850480113E1375F50F31A04C
:1013C0007D141374F40F69F401456FE01FDC7D1484
:1013D0001374F40F61FCCDBFEFE29FD92A89371552
:1013E00001402E84130505C08565B2840146EFF0E7
:1013F000EFDF0D456937135504011375F50F4137BC
:10140000135584001375F50F9D3F1375F40F853F39
:10141000014493170401C18363EC97003715014021
:1014200005468565130505C0EFF04FDC6FE09FD6DC
:101430001305F00FA937B307890088A30504D1BFAE
:10144000EFE21FD3411185451145E13A93070010A2
:101450007C8237150140C1473EC64C008D471305BD
:1014600005803EC4EFF00FCB41016FE0BFD2EFE249
:101470003FD0411185454145EFF0BF9A856793877D
:1014800007807C8237150140C1473EC64C008D471E
:10149000130505803EC4EFF0EFC741016FE09FCF19
:1014A000EFE21FCD411185452145EFF09F9793074E
:1014B0000010371401407C82C1473EC64C008D4766
:1014C000130504C03EC4EFF0EFC4014693050010BD
:1014D000130504C0EFF08FD141016FE0BFCBEFE205
:1014E0003FC9797185452545EFF0BF939147371581
:1014F0000140FC824C0893078004130505C03ECED2
:10150000EFF04FC189450545EFF0AFE19147054444
:101510003ED00810B1473ED422D602D2EFF06FB6CB
:10152000930780117C86680089475C8722C8EFF0AA
:101530006FFB45616FE01FC64111114522C626C4ED
:101540004AC2EFF0AFBA85476311F504371901407D
:10155000AA8401469145130509C0EFF02FC903C7BE
:1015600041883E8411EF0545EF0000660546914530
:10157000130509C0EFF08FC789472382F18819A0AE
:10158000E30C97FE1145EFF04FB83244A2441249E4
:10159000410173002030EFE2BFBD41118545214577
:1015A000EFF03F8885451145EFF09F8993070020B4
:1015B000371401407C82E1473EC64C008D4713053D
:1015C00004C03EC4EFF00FB5930700084C001305AC
:1015D00004C07C82EFF00FB441016FE0BFBBEFE2CB
:1015E0003FB901114D3F371400409307F01D8A8524
:1015F000130504803EC002C223140100230501002C
:10160000EFF0BF8D130504808545EFF03FA0C16763
:10161000938707066C00130504803EC8231B010056
:1016200002C6EFF0FF9213050480A145EFF0BF9FC3
:10163000130504808545EFF07F99854513050480E7
:10164000EFF05F9A05616FE0FFB4411122C42A8474
:1016500008414AC24EC006C6EF409009B787000055
:1016600003A6879683A6C7962A89AE89EF20103DE8
:10167000635F0502B787000083A7C7951CC0B787C3
:10168000000083A547960840EF400000EF40A067A8
:101690009315050137150040C18113050580EFF052
:1016A000FF99B24022441249824941018280B787A2
:1016B000000003A6079783A647974A85CE85EF20AB
:1016C000102DE35EA0FAB787000083A707967DB7C9
:1016D000EFE21FAA797137140140C1472A89FC82C1
:1016E0008D44C1474C08130504C03ECE26CCEFF014
:1016F0006FA20146130504C0C145EFF02FAF854529
:101700002145EFF00FF2854537050800EFF04FF364
:101710008547FC824C08E147130504C026CC3ECE29
:10172000EFF04F9F894491474C08130504C0E482B1
:10173000375400403ECEEFF0EF9D0C10B7070C0081
:10174000130504C04AD03ED402D223160102EFF0A2
:101750001F949307D0137C86680085473EC8448752
:10176000EFF04FD80546130504C093055052EFF033
:101770001F9F8545130504C0EFF01F9D45616FE075
:101780007FA1EFE2FF9E79713714014093070002B9
:101790002A89FC828D44C1474C08130504C03ECE03
:1017A00026CCEFF02F970146130504C093050002E5
:1017B000EFF0CFA385452145EFF0AFE6854537052E
:1017C0000400EFF0EFE793070040FC824C08E1478C
:1017D000130504C026CC3ECEEFF0CF9385679387E8
:1017E0000780FC824C089147130504C03ECE375455
:1017F0000040EFF02F920C10B7070C001305048087
:101800004AD03ED402D223160102EFF05F8893073C
:1018100070137C8685475C87680085473EC8EFF07B
:101820006FCC05461305048093055052EFF03F93AB
:10183000854513050480EFF03F9145616FE09F956A
:10184000EFE21F932A84EFF0FF94930500082285AE
:10185000EFF05F957DD96FE0FF93411122C63754B9
:1018600000409305505213050480EFF05F940DC5BE
:1018700013050480EFF09F929375F50F238CB182CE
:1018800003A5C1881C4D104954498507B3E7C70219
:101890006384D7003105452C324441017300203068
:1018A000411122C63754004093055052130504C01D
:1018B000EFF0FF8F0DC5130504C0EFF03F8E937559
:1018C000F50F238EB18203A501891C4D104954499F
:1018D0008507B3E7C7026384D7003105AD243244DE
:1018E000410173002030EFE2BF880111AA842E84E9
:1018F00009458545EFF0CFD4E084370400404C081B
:101900001305044026CA231E0100231D0100EFF029
:10191000CFDC0546854513050440EFF00FEE930735
:10192000D0027C8685475C87680085473EC8EFF01B
:101930006FBB05616FE01F86EFE29F83B707002052
:1019400083A50716896793870771B3D5F502A94761
:101950003305F502FD15C205C1817D1542054181A2
:1019600059376FE03F83411122C637040040854557
:1019700013050440EFF06FEF01C9854513050440DE
:10198000EFF02FF0EF00902E324441017300203031
:10199000EFE20FFE01112E84AA8485450545EFF084
:1019A0002FCA4C083705004026CAE084231E0100D8
:1019B000231D0100EFF06FD2054685453705004035
:1019C000EFF0AFE39307C0027C868D475C87680029
:1019D00085473EC8EFF00FB1854537050040EFF071
:1019E000EFDE05616FE00FFBEFE28FF8B707002035
:1019F00083A50716896793870771B3D5F502A947B1
:101A00003305F502FD15C205C1817D1542054181F1
:101A100041376FE02FF8854537050040EFF0EFE4E0
:101A200011CD854537050040EFF0AFE5CD2083C6E9
:101A3000418805476394E6002382018873002030C3
:101A4000B7F700E023A20700D9207300203041112E
:101A500022C6373401408545130504C0EFF0EFE09E
:101A600001CD130504C08545EFF0AFE137850000D7
:101A700013058597EF40700C32444101730020300C
:101A80001DC9B296C206C18252A136A10CC509EE8B
:101A900085471CA183A6018493870184368701EBC7
:101AA00054C588C30145828023000500E5B763065D
:101AB000A7005847EDB77D558280054582800DC54A
:101AC00083A701841387018499E305458280D44765
:101AD0006396A6005845D8C7014582806394A70045
:101AE00014C3DDBFB687CDB77D558280EFE24FE8E6
:101AF00003A4018475DC1C2093F7F70F99C75E20BF
:101B000099C3230004001C4482974044E5B783A78F
:101B10000184054691E38280D62381CEBA237D17C6
:101B200042074183BAA3BA234207418319E390A332
:101B3000B6A3DC47C5B7232605000CC150C123243A
:101B40000500054582805C45544118458507B3E78B
:101B5000D702638EE70058451C41BA978CA35C45B9
:101B600058418507B3E7E7025CC505458280795592
:101B7000828018455C45630FF70018451C41BA97F1
:101B80009C239CA11C4558418507B3E7E7021CC56F
:101B900005458280014582805C4518454841998F02
:101BA000AA9733E5A7028280B707002083A707160C
:101BB0000967130707F4B3D7E702C207C18323936A
:101BC000F1842392F1848280B7F700E0D843814604
:101BD000799BD8C303D741843306A70290CBD4CBDB
:101BE00098431367070198C398431367170298C374
:101BF000D843058B75DF9843799B98C38280EFE2C9
:101C00002FD72A841165011185451105EFF06FA1C9
:101C1000930700207C82371501408D473EC44C005D
:101C2000E147130505803EC6EFE0DFCE22C837440A
:101C30000140B70708000C08130504803ECC02CA17
:101C4000231E0100EFF0AFC4854513050480EFF0BB
:101C5000AFCF05616FE00FD4EFE2EFCFB7440140A3
:101C6000AE893289014493840480634524014A8506
:101C70006FE0AFD1930500042685EFF0AFD27DD998
:101C8000B38789008385070026850504C205C181C5
:101C9000EFF04FD0D9BF138781801C43938681B763
:101CA0003E95636BD500B75600209386068063E5AA
:101CB000A60008C33E858280FD57EDBF0397418390
:101CC00081472A97634F070009CD05669306F6FF03
:101CD000B6876358C700AA876305D5009317070125
:101CE000C1833E858280EFE20FC741113724014056
:101CF000AA8944001309010113040440CE852285FA
:101D000095460546EFE0FF8885452285EFE0FF8692
:101D100089452285EFE0FF9365DD2285EFE0FF92A4
:101D200042054185613F8AA08904E31999FC154762
:101D3000814735A0139617001408850736960808C2
:101D400093961700AA96835546FF03D546FF637600
:101D5000B500231AA6FE239AB6FEC207C183E3CBC1
:101D6000E7FC7D1771F728843C8541013E954205CB
:101D7000418105816FE06FC1EFE28FBF0545A53757
:101D8000EF40200AB787000083A58798EF30805383
:101D9000EF400016B787000003A6079983A647996E
:101DA000EF202055B787000003A6879983A6C7991F
:101DB000EF202054EF40801E6FE0CFBDEFE24FBB1D
:101DC00009451537EF40E005B787000083A58798E0
:101DD000EF30404FEF40C011B787000003A60799CE
:101DE00083A64799EF20E050B787000003A6879BA2
:101DF00083A6C79BEF20E04FEF40401A6FE08FB9FA
:101E0000EFE20FB70D45C535EF40A001B7870000E1
:101E100083A58798EF30004BEF40800DB787000017
:101E200003A6079983A64799EF20A04CB787000027
:101E300003A6879983A6C799EF20A04BEF40001611
:101E40006FE04FB5EFE2CFB21145713DEF30707DDD
:101E5000B787000083A58798EF30C046EF40400960
:101E6000B787000003A6079983A64799EF2060482B
:101E7000B787000003A6079B83A6479BEF20604718
:101E8000EF40C0116FE00FB1EFE28FAE1945A13DF9
:101E9000A1679387079C01479306100F92236369FC
:101EA000C5023A85EF304004B787000003A6079AC1
:101EB00083A6479AEF20E043B787000003A6879ADE
:101EC00083A6C79AEF20700EEF40400D6FE08FACF5
:101ED00005078907E314D7FC13050000C5BFEFE22F
:101EE0002FA9797148001306C0028145EFF0CFCECB
:101EF000188293073005370500206317F702988290
:101F00009307C0046312F7020347F102D947631D28
:101F1000F7001306C0024C0013050502EF408025B0
:101F2000054545616FE00FA7B707002003C7C70449
:101F3000130505029387C70418A1983318B1B82375
:101F400038A1B83338B1D82358A1D83358B1F823C1
:101F500078A1F83378B19827DC3718A5A305F502E6
:101F60000145C1B7EFE22F9F9387C189F82FC03F8A
:101F7000AA852207418FE03F1389C1804204418F27
:101F800003C407026204598C2285EF303019B787E9
:101F9000000083A5C7BEEF30206FB787000083A580
:101FA000C7BDAA892285EF30206EAA854E85EF2015
:101FB000D07A83250900EF20507A2320A9001385C9
:101FC000C180EFF08FE86FE04F9CEFE2CF989387EE
:101FD000C189B82B803B2207418FA03B1389C18068
:101FE0004204418FC02B6204598CA285EF3010133C
:101FF000B787000083A507BEEF300069B7870000F0
:1020000083A547BEAA892285EF300068AA854E8540
:10201000EF20B07483250900EF2030742320A9003D
:102020001385C180EFF06FE26FE02F96EFE24F94DF
:10203000938411819C201384C18485C7B707002035
:1020400093870702E83B9C2FA2075D8DEF30705D00
:10205000B787000083A587BAEF30C02608C0238069
:10206000040008409D376FE0EF92EFE2CF8E938738
:10207000C189F82BC03B2207418FE03B1389C18007
:102080004204418F802F6204598CA285EF301009E1
:10209000B787000083A5C7BEEF30005FB787000099
:1020A00083A587BDAA892285EF30005EAA854E856B
:1020B000EF20B06A83250900EF20306A2320A900B1
:1020C0001385C180EFF06FD86FE02F8CEFE24F8A5D
:1020D0001387C1898347C7028346B7020947A2070E
:1020E000D58F6383E70E1384C1896367F7000547C3
:1020F000638DE7066FE00F8A0D47638DE70C11478C
:10210000E39AE7FE138721811C239384418685C3CC
:10211000B706002093860602DC2EB03E9306803E72
:10212000A207D18FB387D702230007009CC0378551
:102130000000130585BBEF40402037150040814566
:1021400013050580EFE09FEF938701869843944045
:10215000050798C3E310D7FA23A00700C13D8D47B8
:10216000A305F4022306040271B713890181834792
:1021700009009384C18585C7B707002093870702AC
:10218000883FBC2FA2075D8DEF30B049B7870000B4
:1021900083A587BAEF30001388C023000900378574
:1021A0000000130505BBEF4040192C2C1C3C884057
:1021B000A205DD8D3C3CC207CD8F4C2CE205DD8DA8
:1021C000EF20B0595D353DB7B787000003A5C7BA0A
:1021D000513B0DB7A13D39BFEFD21FF79384318139
:1021E0009C20138A8185ADCB3704002013040402A0
:1021F0007C24483437890000A2075D8DEF3070429F
:10220000832589BAEF30000C23A4A1841C286834EC
:10221000A2075D8DEF30F040832589BAEF30800A48
:1022200023A8A1843C280838A2075D8DEF30703FB9
:10223000832589BAEF30000923AAA1847C28483875
:10224000A2075D8DEF30F03D832589BAEF3080071E
:102250002320AA00238004009387C189B82F03C9D3
:102260009701C43B22073367270103C9B70183C520
:10227000270203250A0042093367E90003C9C701A1
:10228000A2051384C18962093369E900F82B22078A
:10229000458FE43BC204458F842FE204D98C03C7E9
:1022A0001702D98D03C7370242074D8F83C54702F6
:1022B000E205D98DEF30202C635BA004A6854A850A
:1022C000EF30602B63520502CA852685EF3000652A
:1022D000EF301042B787000003A687BC83A6C7BCB7
:1022E000EF10D07563550502A3050402230604020E
:1022F000EF003074B735000081461306803E9385A9
:10230000051313850195EFF0AFF76FD07FE7CA850E
:102310002685EF30A060EF30B03DB787000003ABFB
:1023200087BC83ABC7BC2A8A5A86DE86AE8AEF108A
:10233000F070635E0500A6854A85EF30205EEF30C1
:10234000303B5A86DE86EF10706F634405043C28EC
:1023500003491401A207B3E72701034934014209E5
:10236000B367F9000349440162093369F900B7878B
:10237000000083A507BC4A85EF30E01F634BA00037
:10238000B787000083A547BC4A85EF3020276358F4
:1023900005008D47A305F40223060402BDB783A9F7
:1023A00081844A85EF30D0342A8B4E85AE8B03ACC6
:1023B0000185B78C0000EF30B03303A60CBD83A6B7
:1023C0004CBDEF10C0695A86DE86EF10306763504F
:1023D00005046285EF30D03103A60CBD83A64CBD49
:1023E000EF20A03C2A86AE865A85DE85EF10106568
:1023F000634FA000B787000003A6879683A6C79601
:102400005285D685EF10B0588947E345A0F8E2859C
:102410004A85EF3040166353A00403AA4185A68580
:102420005285EF3040159147E346A0F65285EF30D4
:10243000302CB787000003A6879683A6C796EF10B7
:1024400000622A8A2685AE8AEF30902A2A86AE86D6
:102450005285D685EF10905EE35DA0F2CE854A8569
:10246000EF30C019E35305EA85472DB7EFD25FD0AF
:10247000EFF09F901384C1899357850048B87CA8DA
:102480009357050161817CB808ACEFF07F979357B3
:10249000850008BC3CAC9357050161813CBC48AC4D
:1024A000EFF0DF919357850048B47CA49357050162
:1024B00061817CB408A8EFF0FF989357850048BC71
:1024C0007CAC9357050161812300A4022C2C682861
:1024D0007CBC183C5C382205A2055D8DD98D7C380A
:1024E000383CC2074207C98F4D8F082C4C2C62051F
:1024F000E205D98D5D8DEF306042B787000083A57E
:1025000007BF2A89EF3020076350A0047C2444349D
:102510004A85A207C58F6434C204C58F0428E2042B
:10252000DD8CB787000083A547BFEF30E015AA8593
:102530002685EF30A03E9357850008B83CA89357F6
:10254000050161813CB848A883C7518889E7EFF04D
:10255000BFC8EFF0BFB76FD0FFC3EFD27FC13785E1
:1025600000001306E02285451305C5DAEF30B04BB5
:102570009387C18903C5B70283C7C702A2075D8DD0
:102580006FD05FC1EFD2DFBE378500001306202277
:102590008545130585D3EF30104903A5418C218172
:1025A000420541816FD01FBFEFD29FBC378500002D
:1025B000130660218545130505D7EF30D046938774
:1025C000C189D85303C58702B787000083A5C7D642
:1025D00021836205598DEF30200BEF30C072420528
:1025E00041816FD03FBBEFD2BFB8378500001306E3
:1025F000A0208545130585DDEF30F0429387C18922
:10260000985303C54702B787000083A5C7D6218327
:102610006205598DEF304007EF30E06E4205418191
:102620006FD05FB7EFD2DFB4378500001306E01F2D
:102630008545130545D0EF30103F9387C189984FEA
:10264000C82FB787000083A5C7D621836205598D9F
:10265000EF308003EF30206B420541816FD09FB394
:10266000EFD21FB1378500001306201F85451305E3
:1026700045CDEF30503B9387C189D84B882FB78722
:10268000000083A5C7D621836205598DEF20D07F36
:10269000EF306067420541816FD0DFAFEFD25FADB1
:1026A000378500001306601E8545130505CAEF3007
:1026B00090379387C189984BC82BB787000083A5B3
:1026C000C7D621836205598DEF20107CEF30A063BF
:1026D000420541816FD01FACEFD29FA93785000022
:1026E0002E841306F0148545130585BFEF30B033F3
:1026F00005472383E1881385019023840186EFF049
:102700000FBC5C245834B7350000A207D98F81462E
:102710001306803E9385256313850193239EF188DC
:10272000EFF00FB66FD01FA7EFD29FA423AEA18604
:1027300015470566B73500002380E188854481464A
:10274000130686BB9385654E13850190238491867D
:10275000EFF00FB3238091906FD0DFA3EFD25FA192
:10276000D425DC35A206DD8E954763FDD70037857D
:102770000000130640128545130545C2EF30B02A0C
:102780006FD05FA1B425BC35A206DD8E9307002073
:1027900063FAD700378500001306B012854513058C
:1027A00045C5E9BF378500001305C5C8EF30F038CF
:1027B000C1BFC16769768146FD17050613970601FB
:1027C00041836364B7003E8582803307D5001823B8
:1027D000B98F214713F81700858363050800B18F6F
:1027E000C207C1837D17420741836DF78506F9B79C
:1027F000EFD21F983715004013050580EFE07F8565
:10280000EF307034EF30B0399307100F3365F502B5
:10281000A94729053305F5026FD0DF97EFD2BF93A3
:1028200003A7C1882A84BE84054693055052631CC1
:10283000A7043755004013050580EFE05F9222851D
:10284000EF100021131905010945EFF0EFB72285BC
:10285000EF10002083A7C1889319050113590901BE
:1028600093D90901014693055052375500406391B1
:10287000870213050580EFE09F8E3305394133351C
:10288000A0006FD09F9037550040130505C075B765
:10289000130505C0CDB7EFD2BF8D370400208347A5
:1028A00004024111130404025C801C302315010052
:1028B000AA84DC803C20AD450A855C813C3023162F
:1028C0000100DC815C205C825C30DC827C205C83EB
:1028D0007C30DC831C245C84930710FDDC848547FA
:1028E0005C85EFF01FED93578500DC858347B402CC
:1028F0004886DC86EFF0DFEFEFF00FAD2685EFF0D6
:10290000FFF16DF93D468A852685EF10400A83A7C1
:10291000C18805469305505237550040639997008A
:1029200013050580EFE0BF8341016FD0BF8613051B
:1029300005C0CDBFEFD2DF833704002083470402F8
:102940004111130404025C801C3023150100AA8489
:10295000DC803C20AD450A855C813C3023160100BB
:10296000DC815C205C825C30DC827C205C837C309F
:10297000DC831C245C84930700FDDC8485475C8534
:10298000EFF03FE393578500DC858347B402488628
:10299000DC86EFF0FFE5EFF02FA32685EFF01FE8D0
:1029A0006DF93D468A852685EF10600083A7C188B2
:1029B000054693055052375500406399970013051B
:1029C0000580EFE0CFF941016FD0CFFC130505C0C2
:1029D000CDBFEFD26FF703C9C500DC350111220965
:1029E0003369F90042091359094193140901C1805F
:1029F000954763FF970037850000A6861306500CA5
:102A00008545130545C2EF30100205616FD04FF7C1
:102A1000B425BC35A206DD8E9307002063FAD700EB
:102A2000378500001306B00C8545130545C5E1BF89
:102A3000AA8902CA02CC231E0100930A4101368AE8
:102A4000370B0020B307DA40C207C18363E1970C5C
:102A50001384C18C1305C400130660028145EFD0B6
:102A60002FF43707002083470702A305240123051D
:102A700004001CA0930707029433939A14001309CF
:102A8000070214B0B42334A0B43334B0D42354A018
:102A9000D43354B0F42374A0F4339C2774B01CA432
:102AA000930700031CB481471384818D63C55709C4
:102AB00093856400860593F5E50F1385C18CEFF0CF
:102AC0005FCF9317850021815D8D8347B9025694AE
:102AD0000AA03CA0EFF0DFD1EFF00F8F4E85EFF0B2
:102AE000FFD36DF913860A019385C18C4E85EF00E3
:102AF000106C83A7C1880546930550523755004096
:102B0000639C370513050580EFE06FE5FDBD1304F9
:102B1000CB08930B84031C40639947015C4001453B
:102B200036C68297B2462390AA002104E3958BFE15
:102B3000890A050A01BF101013F7E70F329713F641
:102B40001700B306F400035747FF11E221838507FE
:102B500098A293F7F70F99BF130505C075B7EFD289
:102B60008FDF370400201304C405AA89AE84328A9B
:102B70001309040398341C406317F7005C40528625
:102B8000A6854E8582972104E31624FF6FD0EFDFE0
:102B9000EFD20FDB41112A8CEF0090676308052A02
:102BA0005145EFF06F821306200381451385C18CD8
:102BB0001384C18CB70D0020EFD08FDE8149814492
:102BC000014A930B1400B78C0000378D0000138B63
:102BD0000D026285EF00D067630A05266285EF006B
:102BE000B0649387C18CD2973EC688A3930A1A001B
:102BF00089476384FA00638E0424182083C70D027A
:102C00006314F710183083471B00631FF70E3785D6
:102C10000000130610278545130545E1EF30A0603D
:102C2000A5476394FA0603D7C1898947631DF7084E
:102C3000382083472B00631BF708383083473B005D
:102C40006316F708582083474B006311F708583084
:102C500083475B00631CF706782083476B0063178C
:102C6000F706783083477B006312F7061824834702
:102C70008B00631DF704378500001306A0288545E7
:102C8000130505E4EF30205A21A08547E3ED97F8BE
:102C9000A9476385FA00894763FF970883D7C189ED
:102CA000094714346392E712130700036399E60699
:102CB000378500001306B02D8545130505EAEF3072
:102CC0008056C5498DA883C78186BDF383C75181CE
:102CD00095CB38303C20F98F5820F98F5830F98F38
:102CE0007820F98F7830F98F1824F98F1307F00FB7
:102CF000639AE700378500001306F0298545130520
:102D0000C5E649B791E085445286DE851385C18CBE
:102D1000EF30404693070003E3FD47EB05AA414728
:102D20006398E602378500001306102E85451305CB
:102D300045ECEF30404F1834C1476312F70CB547EC
:102D400063FF570B8349D4008609C509568AD9B752
:102D5000138706031377F70F0546636DE600378583
:102D600000001306802E8545130585EEEF30A04B3D
:102D7000B549D1B703C751811DCF1307000A130608
:102D8000E02E6389E6041307100A6398E600130631
:102D9000402F85451305CDF21DB7268763F3F40058
:102DA00009479374F70F1306C02F854513854CF51B
:102DB000EF30604791BF268763F3F40009479374AF
:102DC000F70F13067030D5B79307000A639AF60021
:102DD00013060031378500008545130585F079B766
:102DE0009307100A13066031E385F6FAA68763F3AA
:102DF000E400894793F4F70F1306E0317DB7E397BA
:102E00003AF59385DAFF93F5F50F1385C18CEFF052
:102E10005F9A330744018347E7FF0347F7FFA207A1
:102E2000D98F6397A700B2479823D947630AF70061
:102E30000D47A68763F3E4008D4793F4F70FE9B5D8
:102E400056869385C18C6285EFF07FD141016FD0AA
:102E5000EFB2A547E39EFAE2F9B3EFD26FB19387E1
:102E600081889843D566938606186307D7020507BD
:102E700098C337140140856493850480130504804A
:102E80000546EFD0BFB60146938504801305048044
:102E9000EFD0DFB56FD00FB023A00700B707EFBEAC
:102EA00037E700E0938707083CC7E1B7EFD2AFAA46
:102EB00003A5C188B78900005D71938509070D4698
:102EC000EF00F02E1306000581450A85EFD04FADC7
:102ED000B787000083A587BE03A5C1801384C1897D
:102EE000EF20807AEF20105CB78500002A8693855A
:102EF00085F70A85EF30E05203A5C1888A8513065D
:102F00000005EF00D02A1306000581450A85EFD0A1
:102F10002FA968245C343789000022055D8D7C343C
:102F2000832589BAC207C98F082862055D8DEF2005
:102F3000A075EF203057B78500002A86938505F9E4
:102F40000A85EF30004E03A5C1888A851306000567
:102F5000EF00F0251306000581450A85EFD04FA448
:102F600028281C38832589BA22055D8D3C38C20784
:102F7000C98F482862055D8DEF200071EF209052C7
:102F8000B78500002A86938545FA0A85EF306049A7
:102F900003A5C1888A8513060005EF00502113069A
:102FA000000581450A85EFD0AF9F68285C388325EE
:102FB00089BA22055D8D7C38C207C98F082C62054D
:102FC0005D8DEF20606CEF20F04DB78500002A8604
:102FD0009385C5FB0A85EF30C04403A5C1888A8567
:102FE00013060005EF00B01C1306000581450A8595
:102FF000EFD00F9B282C1C3C832589BA22055D8DC0
:103000003C3CC207C98F482C62055D8DEF20C0672C
:10301000EF205049B78500002A86938505FD0A8573
:10302000EF30204003A5C1888A8513060005EF0014
:1030300010181306000581450A85EFD06F960345E9
:103040006402834754023787000022055D8D834761
:1030500074028325C7D6C207C98F0345840262055F
:103060005D8DEF206062EF20F043B78500002A8677
:10307000938545FE0A85EF30C03A03A5C1888A854D
:1030800013060005EF00B0121306000581450A85FE
:10309000EFD00F918347A40203469402B785000046
:1030A000A2075D8E938545FF0A85EF30803703A523
:1030B000C1888A8513060005EF00700F130600050E
:1030C00081450A85EFD0CF8D8347C4020346B40201
:1030D000B7850000A2075D8E938585000A85EF30D5
:1030E000403403A5C1888A8513060005EF00300C23
:1030F00003A5C188938509070D46EF00500B938700
:103100008187902337150140930500101336160070
:103110001305058090A3EFD07F8D61616FD0EF869E
:10312000EFD20F8503A50189EFF09FA66FD08F86A0
:10313000EFD26F82B704002093870402F42FD83FA8
:10314000A206D98E1387418110233971938404021A
:103150009387C18611C6230007001387D6FF9AA361
:103160009A230507420741836306D7009AA321618A
:103170006FD0AF8123900700EFE0DFCC1384C189CB
:10318000135785009357850113062003A300A4025B
:103190002301E402AA891357050181456800A301B0
:1031A000E4022302F40237890000EFC07FFF832589
:1031B00089BA4E85EF20404DEF20D02EB785000014
:1031C0002A86938505066800EF30A02503A5C188EF
:1031D000130620036C00EF00807D83472402034721
:1031E0001402A838A2075D8F8347340203444402C7
:1031F000C207D98F62045D8CDC28A2075D8DEF20A9
:103200005042832589BAEF20E00BA285EF20003FD2
:10321000E35F05F4B735000081467946938545455F
:1032200013850194EFE0DF8513850195EFE03F8979
:103230003DBFEFC2FFF3378700000327C7083705FC
:10324000004081451305054023A6E180EFD01FD83B
:1032500037150040814513050580EFD03FDE6FC074
:103260007FF3EFC2FFF01387A18637090020130612
:1032700009021E23834606026C3E8507C207A2068A
:10328000C183CD8E6385F6001EA36FC0BFF02310EF
:103290000700EFE0BFB29384C1899357850088B8D7
:1032A000BCA8935705016181BCB8C8A8EFE0DFACAA
:1032B00093578500C8B8FCA8935705016181FCB8F5
:1032C00088ACEFE0FFB39357850088BCBCAC935744
:1032D00005016181BCBCC8ACEFE01FBB9357850002
:1032E000A382A4022383F402935705016181A3837F
:1032F000F4022384A402B71401409305001013853F
:1033000004C0EFD0CFED130909021384C1898147AE
:1033100001C99145138504C0EFD0CFEBB337A000AE
:10332000A304F40223050402EFE0DFB19357850004
:103330002301F40293570501A301F40283476402B9
:1033400083445402A300A402A207C58F83447402DD
:1033500061812302A402C204C58F83448402034511
:103360009902E204DD8C8347A902A2075D8DEF205C
:10337000F01EAA852685EF2060286356050283C6C5
:103380005188094713845188639CE600B7350000D3
:10339000814679469385454513850194EFE04FEECC
:1033A00023000400DDB58347890203457902A207A3
:1033B0005D8DEF20B01AAA852685EF20C01B635FC4
:1033C000A000B787000083A707BF23A6F18013855D
:1033D000C180EFE08FA70547A382E188834564029F
:1033E0008347540203455902A205CD8F83457402D9
:1033F00003448402C205DD8D8347690262044D8C5B
:10340000A2075D8DEF209015A285EF20201FE35EBF
:1034100005E60947A382E188EFF0BFE1BDB5EFC241
:103420003FD537050040854513050540EFD01FBA4D
:10343000371501409387C189094705469305001058
:10344000130505C0A385E70223860702EFD00FDA34
:103450006FC05FD4EFC23FD0938621889E2285073C
:10346000C207C1839EA2914663ECF6003715004067
:103470009305400613050580EFD05FBC6FC0FFD0F9
:10348000138421881307600493840187636BF7001A
:1034900083A9040083A5C1804E85EF20C00D63522F
:1034A000A002930700001385C1809CC02310040074
:1034B000EFE0AF9913850194EFE06FE0EFF03FF696
:1034C00075BF4E85EF20D022B787000003A6870581
:1034D00083A6C7056923EF20702C88C01385018758
:1034E000EFE0AF9661BFEFC21FC7138771881C233F
:1034F000011193861700F51714A393F7F70F93069E
:10350000B00F63EDF600138501902384018623003C
:103510000700EFE0CFDA05616FC03FC74146814544
:103520001305E100EFC0DFC7370400208347040222
:1035300013040402DD455C821C30480093847188CA
:10354000DC82FD577C83FD573EC4E9779387F71FE4
:103550007C8683C70188DC8703C7D18983C6C1897C
:103560009387C1892207558FA308E10093568700EE
:1035700038202308D1002309E1003830A309E100F5
:103580005820230AE1005830A30AE1007820230BD9
:10359000E1007830A30BE1001824230CE1009837F8
:1035A000BC27A207D98F13D78700230DF100A30CE6
:1035B000E100EFF00FA093578500A30DF1008347C2
:1035C000B402230EA1002944A30EF100EFF04FA294
:1035D000EFE08FDF1389C18703250900EFF00FA407
:1035E00021E593876188942305476397E60023804C
:1035F00007002380040005B7032509006D464C0031
:103600007D260327090083A7C188054693055052EC
:10361000375500406317F70013050580EFD03FB41E
:10362000DDBD130505C0DDBF7D141374F40F59FC17
:10363000DDB5938741879043938651810506B70591
:10364000002090C3238006009385050203C745022E
:1036500003C535022207498F631EE600EFC25FB142
:1036600023A007001385019385479CA2EFE02FC597
:103670006FC05FB28280EFC2BFAFB70700209387F1
:103680000702B8231384C18938A0B833238E018878
:10369000A38E018838B0D82358A0D83358B0F82367
:1036A00078A0F8339C2778B0370700201307C704A9
:1036B0001CA43C271437A207D58F1CB4A1833CA4BB
:1036C0005C273437A207D58F3CB4A1835CA4EFE01C
:1036D000EFEE93578501135785001CA8935785007B
:1036E00048B478A408B8135705013CA893570501BE
:1036F000618178B43CB848A8EFE00FE893578500A3
:1037000048B87CA89357050161817CB808ACEFE00C
:103710002FEF9357850008BC3CAC9357050161819E
:103720003CBC48ACEFE00FF293578500A300A40225
:103730002301F402935705016181A301F4022302DE
:10374000A402EFE06FF4935785002303F40293572C
:103750000501A303F4023C2803491401A302A402B7
:10376000A207B3E727010349340161812304A402BE
:103770004209B367F9000349440162093369F9005A
:10378000B787000083A547074A85EF103067634B72
:103790000500B787000083A587074A85EF10B05D55
:1037A000635BA00037150140054693050010130523
:1037B00005C0EFD0AFA3B7140140930500101385E7
:1037C00004C0EFD0CFA1814701C99145138504C042
:1037D000EFD04FA0B337A000A304F40223050402E6
:1037E000A3050402230604026FC0DF9AEFC25F98AC
:1037F000EFE0EFEEEFF03FE8B7350000814613064B
:10380000803E9385C5EA13850192EFE06FA7B73537
:103810000000814613064006938505121385019624
:10382000EFE00FA6B7350000F9461306803E9385FA
:10383000A5E513850197EFE0AFA4B7350000930627
:10384000803E1306803E9385252613850191EFE087
:103850002FA3B735000081461306803E93850513DC
:1038600013850195EFE0CFA1EFE04FA86FC09F92C5
:10387000EFC21F900545EFE02F97BD28EFD03FD650
:10388000EFD0BF96EFD0DFBBEFD07FBEEFD0FFA46D
:10389000EFD01FC1EFD0BFC403A5C188B78500001A
:1038A0003D469385C50721220545EFE0EF886FC0AF
:1038B0007F8EEFC2FF8B014405C1002111CC5C411A
:1038C0000D47639EE7003755004093F5F50F13054C
:1038D0000580EFD0FFF6054422856FC0BF8B1147EE
:1038E0000544E39BE7FE3755004093F5F50F1305BC
:1038F00005C0EFD0FFF4CDB7EFC29F87370400209B
:103900001304440C1306800C938501981305C4001E
:10391000EFE06FA2716513050520EFD09FE68544A7
:1039200004A01306C012938581A41305840223A664
:103930008188EFE04FA048507104EFD07FD904A0F8
:10394000014523A881886FC0FF84EFC27F823715AD
:103950000140054693050002130505C0EFD00F890D
:103960006FC05F83EFC2DF803715014001469305CA
:103970000002130505C0EFD06F876FC0BF81EFC293
:103980002FFF371501400546C145130505C0EFD08F
:10399000EF856FC03F80EFC2AFFD37150140014694
:1039A000C145130505C0EFD06F846FC0AFFEEFC2F5
:1039B0008FFA03A7C1882A842E8AB2899384C1888A
:1039C0006311A702EFF07FF801496343390305450E
:1039D000EFE08F9F9C4063968702EFF0BFF86FC0C7
:1039E000CFFA83A70189E391A7FEEFF05FF9E9BF62
:1039F000B3072A018385070022850509EFF07FEBD5
:103A0000E9B783A70189E39C87FCEFF0DFF8C1BF2A
:103A1000814709C91821814711C75C49084D898F21
:103A2000B337F0003E858280EFC28FF441112A84C3
:103A3000A3070100EFF0DFFD19C59305F1001305A1
:103A4000C400EFE00F930305F10041016FC08FF454
:103A5000EFC20FF23105EFE02F946FC0AFF33708DC
:103A6000100001117D183377B80026CA3378D800CA
:103A700093D4450113D34601131E37004EC6135786
:103A8000D5010E089357D60193F4F47F1373F37F97
:103A900006CE22CC4AC893D9F50193DEF6013367EE
:103AA000C701131F350033E80701931F3600338E1B
:103AB00064406380D9196356C0136304031CB706BE
:103AC00080009307F07F3368D800638FF436930744
:103AD000800363C0C735FD4763CDC74713050002A8
:103AE0003305C541B3D7CF01B316A8003399AF0052
:103AF000DD8E33392001B357C80133E926011D8F0C
:103B000033092F41B3372F013306F740931786004F
:103B100063D40724370780007D173374E600630CF5
:103B2000042C2285EF20205E130785FF93070002F7
:103B3000998FB357F9003316E400D18F3319E90098
:103B40006341972A33059740130615007D47634D5F
:103B5000C73813070002118FB356C9003319E900A3
:103B60003397E700558F333920013369270133D666
:103B7000C70081449377790081CF1377F90091478B
:103B80006308F70013074900333927014A963A8939
:103B90009317860063D6071C138514009307F07FE4
:103BA000CE856304F520B70780FFFD17F18F93984A
:103BB000D70113593900A607B3E82801B18313755B
:103BC000F57F9396C7005205F2406244B182FE052C
:103BD000C98ECD8ED2444249B2494685B68505612B
:103BE0008280631E0E0A138314001373E37F63172E
:103BF0000322B367E701B368F801639D041A638782
:103C00000740638608443309FF41B3070741333651
:103C10002F013386C7409317860063D6074C33893C
:103C2000EF41B307E84033B62F013386C740F6892A
:103C300091B76350C00F6300030CB7068000930771
:103C4000F07F3368D800638AF43A9307800363CB2C
:103C5000C713FD4763DFC73513090EFE9307000244
:103C6000B3562801630AFE00130900043309C94151
:103C700033192801B3EF2F013339F0013369D9002B
:103C800031A2B367F801638A071C9307FEFF638CB8
:103C900007389306F07F6309DE1A3E8E0DBDB3052B
:103CA000934063910422B367E701638707329387E8
:103CB000F5FF638107449306F07F638CD520BE85B2
:103CC0009307800363CCB72AFD4763CFB73C9307C4
:103CD00000028D8F3319F700B356BF00B317FF00F2
:103CE0003369D900B337F0003357B7003369F900AF
:103CF0003308E84041ACB367F801638007349307A9
:103D0000FEFF638A07209306F07F6308DE2E3E8E57
:103D10002DBF631E0E149386140093F7E67F639104
:103D20000734B367E7016395042C6380073EB367EC
:103D3000F801638E07303309FF01B3070701333FF2
:103D4000E9013386E7019317860063D70700B707B9
:103D500080FFFD177D8E854493777900E39F07E010
:103D60009317D60193583900B3E8F80093573600FB
:103D70001307F07F638DE404B207B18313F5F47F7A
:103D8000CE8581B53369F801333920017A99B3378B
:103D9000E9013386E70093178600E3DF07FA85041D
:103DA0009307F07F6396F418CE851305F07F814763
:103DB000814801BDC1EB6384083A9316360093171E
:103DC000D8018D82B3E8D700F68993573800B3E75E
:103DD000F800F9DB81451305F07FB707080081483B
:103DE000CDB3370680FF7D167D8E93777900998C51
:103DF000E39507D8B5B74A85EF20E0301307850172
:103E0000FD47E3D5E7D2130685FFB317C900014983
:103E100005BB3369F80133392001DDB13309FF41B6
:103E20003306074133342F0133048640931784004F
:103E300063CD0724B3688900E39308CE81478149A5
:103E400081441DBFE39808F80E059317D7010D8133
:103E5000B3E8A700935737009DBF0E059317D7010E
:103E60000D81B3E8A700F2849357370011B73305EB
:103E7000934063820412B70680009307F07F558F4A
:103E8000630DF32E9307800363CBA720FD4763C325
:103E9000A72A93070002898F3319F700B356AF00A2
:103EA000B317FF003369D900B337F0003357A700C9
:103EB0003369F9003A987E99B337F90133860701DF
:103EC0009A84D1BDB70680009307F07F558FE31920
:103ED000F3DE931736008D839318D801B3E81701EA
:103EE000F68993573800E5B5130715FE93060002CF
:103EF00033D7E700630AD600930600043386C64032
:103F00003396C7003369C900333920013369E900AA
:103F10000146814491B53309FF01B30707013336E8
:103F2000E9013E96931786008544E3D707E289446A
:103F3000B70780FFFD17F18F135719001379190088
:103F4000336927019398F70133E9280113D6170045
:103F500015B113090EFE93070002B3562801630A38
:103F6000FE00130900043309C94133192801B3EFD6
:103F70002F013339F0013369D90059B63369E701AC
:103F80003339200133892F41B3B72F013306F8406D
:103F90009A84F689A5BEB367E70163820718930781
:103FA000F5FF6384071C9306F07F6304D5123E85FA
:103FB000D1BD93070002B387C741B316F800339908
:103FC000FF0033D6CF01D18E33392001B357C8015A
:103FD00033E926013E975DBB931736008D83931816
:103FE000D801B3E81701AE8493573800F68949B376
:103FF000EDC33369F801E31F09DC0E059317D70100
:104000000D81B368F50093573700D1B36381080E73
:10401000931636009317D8018D82B3E8D700F6893E
:104020009357380091BB3309FF41B3070741333F32
:104030002F013386E7418544D1BC0E059317D70184
:104040000D81B368F500F2849357370015B30E0560
:104050009317D7010D81B3E8A7009357370029BB09
:104060009307F07FE382F6D43309FF013336E90189
:10407000B3070701B2979398F7011359190033E971
:10408000280113D61700B684C1B93389EF4133072D
:10409000E84033B62F013304C740F68949B4336989
:1040A000E7013339200101BD938705FE9306000225
:1040B000B357F700638AD50093060004B385B64072
:1040C0003317B700336FEF003339E0013369F9007C
:1040D00055BD931736008D839318D801B3E81701A7
:1040E00093573800EDB1B368C900E39708C681471C
:1040F000814959B13389EF41B307E84033B62F0105
:104100003386C740F689854411B493163600931759
:10411000D8018D82B3E8D70093573800B1B9931610
:1041200036009317D8018D82B3E8D700AA8493573D
:1041300038003DB9930705FE93060002B357F70018
:10414000630AD500930600043385A6403317A70001
:10415000336FEF003339E0013369F900A9BB8145C2
:104160001305F07FB7070800A9BC3309FF01B307A7
:1041700007013336F9013E9675B39316360093174F
:10418000D8018D82B3E8D7009357380089B113D78F
:104190004501B7071000FD1713D846011377F77FC5
:1041A0009308F07F33F3B7002A8EF58FFD81B28E2E
:1041B0001378F87FFD8263081703630018030DEB83
:1041C000B368A300631408005D8E29CA63850804E0
:1041D0006388D502054595ED8280B3E8C700E3808A
:1041E00008FE795582803365A30065FD630CE80203
:1041F000631408005D8E79DEE39ED5FCE34CE8FC99
:1042000063480701E3E867FC6303F302637FF3009D
:1042100081E57D558280F5DE054582800145E39B81
:1042200008FA82805D8E69DA6DBF01458280E3E322
:10423000CEFB0145E372DEFBE5F1E1BF13D745019B
:10424000B7071000FD1713D846011377F77F9308BF
:10425000F07F33FEB700AA8EF58FFD81328F137881
:10426000F87FFD82630E1703630D180129E3B3681D
:10427000AE00631F08005D8E01EE0143638C0804ED
:1042800021A8B3E8C7000943639608046DD305A0CD
:10429000638408046385D50205438DCD7D531DA835
:1042A000B368AE00094363970802630AE802631427
:1042B00008005D8E75D2E391D5FEE34FE8FC6349BB
:1042C0000701E3EBC7FD630FFE0001436374FE00CB
:1042D000F1D505431A858280EDFE7D53E5BF5D8EE5
:1042E00079DACDBFE36ADFFB0143E3F5EEFFF5F1D9
:1042F00075B739714AD813D945014ED652D456D222
:104300009399C50006DE22DC26DA5AD05ECE1379F8
:10431000F97F2A8A93D9C90093DAF501630D090E52
:104320009307F07F6306F9181354D5018E09B3691A
:1043300034013704800033E48900931435001309F5
:1043400019C08149814B13D74601139AC6001377D0
:10435000F77FB285135ACA0013DBF601630B07100F
:104360009307F07F6303F7049357D6010E0A33EAED
:104370004701130717C0B7078000B367FA0093150A
:1043800036003A99814833C76A01BD463A85130819
:10439000190063E83617174600001306A6CF8A09EE
:1043A000B29983A60900B2968286B367CA00130940
:1043B000F97F6399071293E9290081458948E1B79C
:1043C00001479307F07F3704080081443204D20785
:1043D00031807E075D8C598CA285F250625426850F
:1043E0004259D254B259225A925A025BF24B21617D
:1043F00082805A853E84AE84C68B8947638DFB0ECE
:104400008D47E38FFBFA85472A87639EFB388147F8
:104410000144814465BF33E4A90061C036C632C49B
:10442000638C092A4E85EF10104E2246B246AA87A9
:10443000130755FF7544938487FF198CB39999002E
:1044400033548A0033643401B3149A0013D74601FD
:104450001309D0C0139AC6001377F77F3309F940C8
:104460008149814BB285135ACA0013DBF601E31967
:1044700007EEB367CA00B1C7630F0A22528532C480
:10448000EF10704822462A87930655FFF54793059B
:1044900087FF958F331ABA00B357F600B3E7470189
:1044A000B315B6003309E9401309D9C08148E1BD0D
:1044B00033E4A90001ECA14981441309F07F894B41
:1044C00059B593E919008145854875BD4E84AA8484
:1044D000B1491309F07F8D4BBDB591498144014924
:1044E000854B95B593E93900D2878D4869BD8947D9
:1044F0005685E397FBF02A879307F07F01448144B8
:10450000F1B5C16E1386FEFF93D6040113DE0501DB
:10451000F18CF18D338695023383B60293580601F0
:1045200033059E021A95AA98B382C60363F3680006
:10453000F692C16F1383FFFF33F5670093D3070132
:10454000B3F76800C207337366003E9333069502E3
:1045500093D80801B387A602135F0601B3849302C0
:10456000BE94FA94B38E760263F3F400FE9E416A21
:104570009307FAFF935F0401B376F400B3F9F400F4
:104580007D8EC1803384D502C209338FD401B299A4
:10459000CE98B307DE02935E0401B385BF02AE97E7
:1045A000BE9E330EFE0363F3BE00529EC167938529
:1045B000F7FF33F6BE006D8C4206229693DE0E01A5
:1045C000B305D502769E3385AF0213D40501B386B9
:1045D000D302AA96A296B38FF30363F3A600BE9FFD
:1045E00041657D15B3F7A600C2076D8DAA97B38507
:1045F0005800B3B93501FA97B2953384370133B611
:10460000C500B30EC4013385CE0033343401B3B7D3
:10461000E701C18F33BECE0113D406013336C50086
:104620003E943366CE009394950032947E94B3E426
:104630006400260493567501B3349000DD8193170E
:104640009500CD8C558CDD8C9317740063DB0700CF
:1046500093D7140085889316F401DD8CD58C0580E2
:1046600042899307F93F6359F00893F6740081CEAD
:1046700093F6F40011466388C60093864400B3B4F1
:1046800096002694B6849316740063D80600B70784
:1046900000FFFD177D8C930709409306E07F63CFF1
:1046A000F60E93D634009314D4012604D58C3180B1
:1046B00093F7F77F21BB328532C4EF10D0249306E5
:1046C0005501F147130705022246E3D1D7DC6115F6
:1046D000B317A6008145F9B3EF10F0221307550177
:1046E000F145930705022246B246E3D5E5D46115AC
:1046F0003314AA00814499BB85469D8EB1E7130906
:10470000E941B3972401B3D4D40033192401B3375A
:10471000F000B3649900DD8C93F77400B356D400B5
:1047200081CF93F7F40011466388C7009387440054
:10473000B3B49700A696BE849397860063D8070407
:1047400085470144814459B113068003E341D6CC27
:104750007D46E356D6FA0556B307F64093050002A8
:104760003356F4006387B6001309E943B3172401F5
:10477000DD8CB3349000D18C93F67400014499CA57
:1047800093F7F40011468146E392C7FA139496001A
:104790003180F6068D80D58C81470DB99307F07F67
:1047A0000144814425B142896DBD370710007D1752
:1047B00001113373B70093D84601758F935ED6010C
:1047C00022CC26CA0E0393D445019357D5010E0778
:1047D00006CE4AC84EC693F8F87F130EF07F33E733
:1047E000EE0093F4F47F13D4F50133E36700131F55
:1047F0003500FD82931E36006380C81993C61600EB
:10480000B38514416305D4126351B018638B081A41
:10481000B70780005D8F6381C4599307800363C429
:10482000B734FD4763C5B748930700028D8FB3D9EE
:10483000BE003318F700B39EFE00336838013357CB
:10484000B700B339D001336838013303E340B3090B
:104850000F41B3373F013306F3409317860063D30C
:104860000724370980007D1933792601630F092C4D
:104870004A85EF105009130785FF93070002998FAF
:10488000B3D7F9003316E900D18FB399E900634437
:10489000972A058F13061700FD4663C5C63A13070E
:1048A0000002118FB3D6C9003398E9003397E700AF
:1048B000558F33380001B369070133D6C7008144EF
:1048C00093F7790081CF93F6F90091476388F6005A
:1048D0009386490033B836014296B689931786000D
:1048E00063D6071C138714009307F07F05886306BF
:1048F000F720B70780FFFD17F18F1398D70193D9E1
:104900003900A60733683801B1831377F77F939690
:10491000C7005207B1827E04D98EC18EF240624434
:10492000D2444249B2494285B685056182806356C8
:10493000B00A638A0812B70780005D8F6387C42DB1
:104940009307800363C7B718FD4763D2B73C13884A
:1049500005FE93070002B3590701638AF500930728
:104960000004B385B7403317B700B3EEEE00333819
:10497000D0013368380195A2B367D70193851480BD
:1049800099E393C61600630AD404D1E19387140017
:1049900093F7E77F6399071EB367E3013368D70195
:1049A000639204166382073C6316084213183500AD
:1049B0009316D3011358380033E806019357330098
:1049C00019A2B367D7016385071A9387F5FF638B35
:1049D000073A638CC523BE8589B56399051C938608
:1049E000140093F7E67FC1EFB367E30163900436E9
:1049F000638D0744B367D701639407460E05131808
:104A0000D3010D813368A800935733006DA8B38597
:104A1000984063970420B367E301638D0730938761
:104A2000F5FF638907401305F07F6383A520BE85EA
:104A30009307800363C2B72AFD4763C8B73C930757
:104A400000028D8F3318F3003356BF00B317FF00F9
:104A50003368C800B339F0003353B300336838010A
:104A600033076740B5ACB367D701638307109387FB
:104A7000F5FF638F071E6380C52FBE85D1B59307F1
:104A8000F07F638BF606FA9E33B6EE01B307E300C0
:104A9000B2971398F70193DE1E00B369D80113D6BD
:104AA0001700B68493F77900E39F07E09317D601C8
:104AB00013D839003368F800A685935736001307DA
:104AC000F07F6380E506B207B18313F7F57F0588B1
:104AD0003DBD3367D7013338E000B309E801B3B710
:104AE000E9013386670093178600E3DD07FA850442
:104AF0009307F07F639CF41805881307F07F8147C4
:104B0000014831B5639107106301083C1318360062
:104B10009317D701135838003368F8003684935739
:104B20003700B367F800E9DB01441307F07FB707EC
:104B300008000148E9BB370680FF7D167D8E93F79C
:104B40007900998CE39107D895B74E85EF10A05B5B
:104B500013078501FD47E3D2E7D2130685FFB3971C
:104B6000C90081492DB33368D70133380001C5B17D
:104B7000131835009317D301135838003368F80021
:104B8000935733002DBFB309DF413309E340333678
:104B90003F013309C9409317890063CA072033E8EE
:104BA0002901E31508CC8147014431BFB385984002
:104BB00063810414B70680009307F07F3363D3004A
:104BC0006381F8209307800363CCB722FD4763C954
:104BD000B72C930700028D8F3318F300B356BF0034
:104BE000B317FF003368D800B339F0003353B30074
:104BF000336838011A97B309D801B3B7D90133869E
:104C0000E700C684CDB5E31108F2131835009317F9
:104C1000D301135838003368F8009357330011B7A5
:104C2000370580009307F07F3363A300E392F8E039
:104C30000E061318D7010D823368C800935737004A
:104C40003684C5B505179306000233D7E700630A1B
:104C5000D600930600043386C6403396C700B3E9F6
:104C6000C90033383001B369E800014681441DBDF5
:104C7000B309DF01B307E30033BFE9013386E7017E
:104C8000931786008544E3DF07E08944B70780FF78
:104C9000FD17F18F13D7190013F8190033680701B6
:104CA0009399F701B3E9090113D6170011B91388D5
:104CB00005FE93070002B3590701638AF5009307C5
:104CC0000004B385B7403317B700B3EEEE003338B6
:104CD000D00133683801A5BE3363E3013338600087
:104CE000B3890E41B3B73E013306F740C68436841C
:104CF000ADB6B367E301638707189387F5FF638C4D
:104D0000071C9306F07F638ED50ABE8565BD9307A9
:104D100000028D8FB3D9BE003318F700B39EFE009A
:104D2000336838013357B700B339D00133683801DD
:104D30003A9365B3131836009317D7011358380008
:104D400033E8070136849357370095BBBDCB3367F3
:104D5000D701E31B07DC0E051318D3010D8133685F
:104D6000A8009357330075BBE30F08E21318360011
:104D70009317D701135838003368F80036849357D7
:104D8000370091B3B309DF41B307E340333F3F013D
:104D90003386E7418544D1B4131835009316D30107
:104DA0001358380033E80601935733009DBBB3898D
:104DB000EE413306674033B93E013309264136845C
:104DC00075B40E061318D7010D823368C8009357C7
:104DD000370081BBB309DF41B307E34033363F01FE
:104DE0003386C7409317860063D7070AB389EE411D
:104DF000B3076740B3BE3E013386D7413684C9B49A
:104E00003363E30133386000FDB3138805FE930775
:104E10000002B3590301638AF50093070004B385C8
:104E2000B7403313B300336F6F003338E00133689A
:104E300038017DB5B389EE41B3076740B3BE3E018B
:104E40003386D7413684854409BC1318360093173E
:104E5000D701135838003368F80093573700A5B1CD
:104E6000B309DF01B307E30033BFE9013386E7018C
:104E700093178600E3D807C2B70780FFFD177D8E22
:104E800085440DB10E061318D7010D823368C80092
:104E9000935737002DB133E8C900E30608D019B1A4
:104EA000138805FE93070002B3590301638AF500D6
:104EB00093070004B385B7403313B300336F6F001B
:104EC0003338E001336838013DB301441307F07F04
:104ED000B70708002DBCB309DF01B307E300B3BE79
:104EE000D9013386D70169BB411106C622C426C247
:104EF0000DCD9357F541B3C4A7009D8C2A84268518
:104F0000EF1060209306E041898EA9477D8093F6DB
:104F1000F67F63CDA7022D47098FB3D7E40055056F
:104F2000B207B394A400B18329A00144814681470C
:104F30008144B207D206B1837E04D58FC18FB240BF
:104F400022442685BE859244410182805515B3973F
:104F5000A400B207B1838144E9BF41113707800043
:104F60007D1713D8750126C2935475013373A700BA
:104F700093F4F40FB376B7004AC01378F80F1359BF
:104F8000F50106C622C4FD819A8726854A86131E2E
:104F90003300939E3600B3880441630AB90E635010
:104FA000100D630408149307F00F638BF414B70714
:104FB0000004B3EEFE00ED4763C11729930700021A
:104FC000B3871741B397FE00B3D81E01B337F00083
:104FD000B3E7F800B307FE4013975700635E071866
:104FE000370400047D147D8C2285EF10C0116D15EF
:104FF000B317A4006348951A058D13041500130711
:105000000002018F3397E7003337E000B3D7870002
:10501000D98F814413F7770019C713F7F70091462A
:105020006303D700910713975700635B0714850448
:105030001307F00F4A866383E4169A07A58313F5D6
:10504000F40FB2402244A6079314750113D59700BC
:10505000458D7E0692440249518D410182806399BB
:10506000080A138714001377E70F63170714639078
:105070000422630D0E1EE3860EFCB307DE41139778
:10508000570063500722B387CE412E8961B7635C16
:10509000100B630E08089307F00F6383F406B7073D
:1050A0000004B3EEFE00ED4763C9171F930700022B
:1050B000B3871741B397FE00B3D81E01B337F00092
:1050C000B3E7F800F297139757006357070A850470
:1050D0001307F00F6384E40CB706007E13D71700A4
:1050E000FD16858B758FD98F35B7638D0E08FD182A
:1050F000B307DE41E38208EE9307F00FE39DF4EA85
:10510000630D030801461305F00FB707400015BFF4
:1051100033079840EDE863020E147D176308071803
:105120009307F00F6319F80E2E893683D1BF638B76
:105130000E04FD18B307DE01E38708F89307F00FAC
:10514000E393F4F675BF63950808850413F7E40F3D
:105150006313071263170510630F0E14E3830EEE3B
:10516000B307DE01139757008144635707003707E1
:1051700000FC7D17F98F854413F77700E31F07E8DC
:1051800013D337009307F00FE38CF4F693179300D3
:10519000A58313F5F40F4A866DB54A861305F00F03
:1051A000814745B5370700FC7D17F98F13F7770066
:1051B000898CE31407E6E9B73304DE419317540002
:1051C00063C3070CE31204E201460145814795BD24
:1051D00033079840ADC49307F00FE308F8F4B7071E
:1051E0000004336EFE00ED4763CCE70C930700022A
:1051F000998FB317FE003357EE00B337F000D98F05
:10520000F697C284C9B59307F00FE30FF8F0B7071C
:105210000004336EFE00ED4763C3E7089306000207
:10522000998EB316DE00B357EE003337D000D98F16
:10523000B387FE40C2842E8945B3854761BB630EA8
:105240000E067D17B307DE01C284E30E07E693075F
:10525000F00FE31AF8F8368365B53683C2842E89D9
:1052600015B7E3040EECE38D0EE869BD638D0E0205
:105270002E86B687F9B39307F00FE381F4F2B307F4
:10528000DE018583D5BD3384CE412E89B1BBE31CBD
:105290000EFCE3890EE62E8949BD854725B5854775
:1052A00041BFE39B07EC0146814761BBB387CE4119
:1052B000C2842E8915B3B68769B33683C284D9B543
:1052C00085473DBF3971935775014AD856D25ECE96
:1052D000931A95001359F50106DE22DC26DA4ED624
:1052E00052D45AD093F7F70F93DA9A00CA8B63829D
:1052F00007121307F00F6384E7128E0A37070004C2
:10530000B3EAEA00138A17F80144014B93D77501F9
:105310009394950093F7F70FA58093D9F501FDC7F6
:105320001307F00F6387E7028E04938717F8370798
:105330000004D98C330AFA408146558C1737000097
:10534000130747D90A043A941C4033493901BA97E4
:105350008287130A1AF0F9E88946558C173700003E
:10536000130747DB0A043A941C4033493901BA97C2
:10537000828701491307F00FB70740001395970084
:10538000F25062549317770125817E095D8D336554
:105390002501D2544259B259225A925A025BF24B19
:1053A000216182801307F00F8147C9BFA68ACE8B87
:1053B000368B8947630BFB1A8D47E30CFBFA854755
:1053C000630AFB0A1307FA0713F91B006357E0127D
:1053D00093F77A0099C793F7FA0091466383D70051
:1053E000910A93974A0063D90700B70700F8FD17A1
:1053F000B3FAFA0013070A089307E00FE3C4E7FAC9
:1054000093976A00A5831377F70F8DBFB9E485469C
:10541000A9B763940A021144014A054BC5BD6399BB
:105420000A002144130AF00F094BCDB58D4631B760
:105430003144130AF00F0D4BD1BD56852EC6EF0037
:10544000904C9307B5FFB39AFA009307A0F8338AFC
:10545000A7400144014BB24555BD2685EF00B04A37
:105460001307B5FFB307AA00B394E400138A6707D4
:105470008146E1B513F91B000147814701B7416639
:10548000139554007D1693570501698E63FA9A0AA5
:10549000B3D5FA027D1AD68601473388C502B3F622
:1054A000F602C206558F637B07012A979386F5FFA4
:1054B0006368A70A6376070BF9152A973307074134
:1054C000B356F7023377F702B38AC6029317070180
:1054D00063FB5701AA971387F6FF63E1A70863FFF1
:1054E0005707F916AA97C205B38A5741D58DB33A23
:1054F0005001B3EA5501CA8BF1B58546998E11C7A3
:105500006D4601478147E34BD6E6130AEA09339A11
:105510004A01B3D7DA00B33A4001B3E7570113F7B2
:10552000770019C713F7F70091466303D700910777
:1055300013975700634807029A07A58301473DBDAB
:1055400093D61A00B3D5F6021397FA014183338834
:10555000C502B1B7CE8B368B814AA1BDBA8661B781
:10556000B685A9BF0547814711BD13F91B00130775
:10557000F00F814721B593567501B7078000FD17DD
:1055800013D6750193F6F60F1308F00FB3F8A700C2
:105590001357F501ED8F1376F60FFD816381060336
:1055A000630C06018DE211E2B1C3638E080263054C
:1055B000B70405451DE78280F5D779558280E39EC3
:1055C00008FE6309D60211E2EDD7E314B7FEE34209
:1055D000D6FE63C7C600E3EE17FD0145E3FDF8FC08
:1055E00001E77D558280F5DD054582800145E39226
:1055F00008FC8280F9DBD1B78146E1BF9356750183
:10560000B7078000FD1713D6750193F6F60F130840
:10561000F00FB3F8A7001357F501ED8F1376F60FCF
:10562000FD81638706036309060185EA11EA89EBB8
:105630000145639B080082800945F5FFE5DA31A842
:10564000638C08026300B704054575D77D558280D9
:105650000945639808026304D60211E2F5D7E31501
:10566000B7FEE343D6FE63C7C600E3EF17FD01456F
:10567000E3F3F8FC19E3D9BFF1D905458280E5D3FE
:10568000828082808146C5B7797122D41354750116
:105690004ECE52CC9319950006D626D24AD056CA81
:1056A0005AC81374F40F93D99900135AF50169C4B9
:1056B0009307F00F6308F40E93973900370700043F
:1056C000B3E9E700130414F88144014B13D77501C3
:1056D000939A95001377F70F93DA9A0013D9F5018F
:1056E00045CF9307F00F630CF7028E0A130717F8E4
:1056F000B7070004B3EAFA003A94014633452A0199
:10570000BD47AA869305140063E29710173700007F
:10571000130747A48A04BA949C40BA97828713045B
:10572000F40F63980A0C93E424000946C1BF0145B5
:105730001307F00FB7074000B2502254A6075E07C8
:10574000A5837E05D98F92540259F249624AD24A02
:10575000424B5D8D45618280CA86D689328B8947EE
:105760006301FB0A8D47E304FBFC85473685631222
:10577000FB1A01478147C9B7639E090413D7750116
:10578000939A95001377F70F91440144054B93DAF0
:105790009A0013D9F50131F7639D0A0093E41400D0
:1057A0000546A9BF63930902A1441304F00F094BF6
:1057B00031BF5685EF0030159307B5FF098CB39ABA
:1057C000FA001304A4F8014615BFB1441304F00F06
:1057D0000D4BEDBD4E852EC6EF00F0129307B5FFC1
:1057E0001304A0F8B399F900098C8144014BB24528
:1057F000F1BD93E434000D4611B78947D286E31317
:10580000FBF636851307F00F81473DB741639306DA
:10581000F3FF13D6090193D80A01B3F7D900B3FAFD
:10582000DA0033885703B389F80213570801B30A23
:105830005603D6994E9733061603637357011A968B
:10584000C167FD17B376F7003378F800C206C29639
:105850009399660093570701B3393001E982B297F3
:105860009A07B3E6D900B3E9D7009397490063D903
:10587000070013D7190093F71900B369F7002E84B6
:105880001307F4076350E00493F7790099C793F77F
:10589000F90091466383D70091099397490063D932
:1058A0000700B70700F8FD17B3F9F900130704085C
:1058B0009307E00F63CBE70493976900A583137701
:1058C000F70F9DBD8547B386E74011C76D46014779
:1058D0008147E343D6E61307E4093397E9003337FA
:1058E000E000B3D7D900D98F13F7770019C713F7A2
:1058F000F70091466303D700910713975700634C55
:1059000007009A07A583014705BD1307F00F8147DC
:1059100025B52E84B5B70547814739BD37078000C7
:1059200041117D179356750113D87501B377A70000
:1059300093F6F60F935EF5013376B70026C24AC0A0
:105940001378F80F06C622C41303F00F3E8E368973
:10595000F684139F3700FD8113153600B388064186
:105960006302681093C51500638CBE106354100D5C
:10597000631008106304051EFD18B307AF4063866B
:1059800008029307F00F6388F616ED4763C71729DF
:1059900013070002330717413317E500B35715010A
:1059A0003337E000D98FB307FF4013975700635197
:1059B000071A370400047D147D8C2285A9276D15F4
:1059C000B317A400634E251B3305254113041500AE
:1059D00013070002018F3397E7003337E000B3D796
:1059E0008700D98F014913F7770019C713F7F7001C
:1059F00091466303D700910713975700635E07141E
:105A0000930619001307F00F93FE14006386E61641
:105A10009A07A58393F6F60FA607B240224413D542
:105A20009700DE069397FE01558D924402495D8DE5
:105A3000410182806392080A138716001377E70FEB
:105A4000631B07146394062263020F2071D5B3070A
:105A5000AF401397570063550722B307E54101494B
:105A6000AE8451B7E30005F0638ABE0AE35410FD2B
:105A70009307F00F6381F608B70700045D8D31B717
:105A8000635E1009630108089307F00F6385F6064B
:105A9000B70700045D8DED4763C0171F13070002B1
:105AA000330717413317E500B35715013337E000CB
:105AB000D98FFA9713975700635C070805091307F6
:105AC000F00F630BE90AB706007E13D71700FD1627
:105AD000858B758FD98F01BF3307D840639506102A
:105AE000630D0F147D176303071A9307F00F6314F8
:105AF000F810AE84328E630F0E06814E9306F00FBF
:105B0000B707400011BF39C9FD18B307AF00E383E1
:105B100008FA9307F00FE390F6F8F1BF63990808CD
:105B2000138916001377E90F63160712639B06109B
:105B300063030F16E30205EEB307AF001397570098
:105B4000014963570700370700FC7D17F98F0549A6
:105B500013F77700E31C07E813DE37009307F00F15
:105B6000E30BF9F893179E00A5839376F90F93FE44
:105B700014005DB593FE14009306F00F814769BDD4
:105B8000370700FC7D17F98F13F777003309A94019
:105B9000E31E07E4D1B73304AF409317540063C347
:105BA000070CE31C04E0814E81468147B5B53307FD
:105BB000D840B5C69307F00FE30EF8F2B70700041C
:105BC000336FFF00ED4763CDE70C93070002998F19
:105BD000B317FF003357EF00B337F0005D8FB30703
:105BE000A7004289C1BD9307F00FE304F8F0B7079F
:105BF0000004336FFF00ED4763C2E708930700021C
:105C0000998FB317FF003357EF00B337F000D98FE8
:105C1000B307F5404289AE8449BB854769B3630E3B
:105C20000F067D17B307AF004289E30507E8930726
:105C3000F00FE319F8F8328E7DBD328E4289AE84C2
:105C400031BFE3090FEAE30805EA45BD0DCDAE8E8D
:105C5000B287D9B39307F00FE300F9F2B307AF00AF
:105C60008583FDB53304E541AE8481BBE31D0FFCA4
:105C7000E30505E8AE84BDBD854725BD854749BF21
:105C80000149E39707EC814E814779B3B307E541BA
:105C90004289AE8419BBB28741B3328E42897DBD41
:105CA000054735BF37068000135775019307F6FF88
:105CB0001377F70F9305E007B3F6A7009357F501A5
:105CC00063FCE5009305D00963FAE5003705008021
:105CD0001345F5FF3E95828001458280930550096A
:105CE000D18E63CDE500130660093307E64033D754
:105CF000E6003305E040F5F33A8582801307A7F606
:105D00003397E600FDB713577501370680009307F8
:105D1000F6FF1377F70F9305E007B3F6A700935745
:105D2000F501014563F4E50099C382808280930701
:105D3000E0097D55E3EBE7FE93055009B3E7C600A4
:105D400063D7E5001307A7F63395E70082801305B4
:105D500060093307E54033D5E7008280411106C66C
:105D600022C426C20DCD9357F54133C4A7001D8C24
:105D7000AA842285492E9307E0093387A740930719
:105D80006009FD8063CCE702A1469377F70F63D5E6
:105D9000A60061153314A4002604258021A08144A7
:105DA00081470144260413559400B2402244DE0783
:105DB000FE045D8D458D92444101828093079009D8
:105DC00063DDE7009307B5019546B317F400898EAC
:105DD0003354D400B337F0005D8C954763D6A700E9
:105DE0009307B5FF3314F400B70600FCFD16937754
:105DF00074003376D40085C39377F4009145638CA7
:105E0000B70011069317560063D707009307F009F0
:105E1000758E3387A7401314660025809377F70F9C
:105E200051B7411106C622C415CD2A84E92C930727
:105E3000E0093387A7409307600963C0E704A146E0
:105E40009377F70F63D5A60061153314A4002604D9
:105E50002580260413559400B2402244DE075D8D50
:105E6000410182800144260413559400B24022442B
:105E70008147DE075D8D410182809307900963DDD4
:105E8000E7009307B5019546B317F400898EB33741
:105E9000F0003354D4005D8C954763D6A700930778
:105EA000B5FF3314F400B70600FCFD1693777400B9
:105EB0003376D40085C39377F4009145638CB700A3
:105EC00011069317560063D707009307F009758EE4
:105ED0003387A740131466002580260413559400C9
:105EE000B24022449377F70FDE075D8D4101828037
:105EF000135775011377F70F41119307170022C449
:105F000026C21314950006C693F7E70F2580935415
:105F1000F50185C793573400130707387604B20795
:105F20005207B1831395F401D98FC98FB2402285EE
:105F300022449244BE854101828005EB39C422850A
:105F4000D922A94763C6A7042D47098F9307550196
:105F50003357E4003314F4009317C7001307903845
:105F6000098FB1831377F77F5DBF01CC13573400DE
:105F7000B7070800D98FB2077604B1831307F07F03
:105F800079BF1307F07F814759BF0147814741BF60
:105F9000130755FF3317E40001447DBF93D6450135
:105FA0009397C50093F6F67FB183138616008E078C
:105FB0001357D5011376E67FFD815D8F9318350069
:105FC00035CE138806C89307E00F63DD07018147CC
:105FD000139597009306F00FDE062581FE05558D7B
:105FE0004D8D82806355000B931765000E07B33704
:105FF000F000D98F93D8D801B3E7170113F77700D2
:106000006301071013F7F70091466303D700910768
:10601000370700047D8F75C7130718001306F00FAC
:106020009376F70FE305C7FA9A07A58313959700B0
:10603000DE062581FE05558D4D8D8280B3671701E3
:1060400099EE85CF95479A07A5831395970093F608
:10605000F60FDE062581FE05558D4D8D8280A5DB70
:10606000B7074000139597009306F00FDE068145B1
:106070002581FE05558D4D8D8280814713959700B2
:106080008146DE062581FE05558D4D8D8280A55702
:106090006348F804F94737068000B38707417D4518
:1060A000598E6351F50479573307074113050002F0
:1060B0003357E6006388A700938626CAB316D60036
:1060C000B3E8D800B3371001D98F13F77700014830
:1060D00015FB139757008546E34807F48146A5B79B
:1060E00081468DB7938626C83397D8003337E000B2
:1060F000B316D600B3D8F800B367D700B3E7F800FB
:10610000E9B7C28689B7C167637CF5029307F00FD0
:106110001307000263EBA700972700009387870708
:10612000AA9788233305A740828021819727000002
:1061300093874706AA97882361473305A740828043
:10614000B7070001636DF500618197270000938711
:106150006704AA97882321473305A740828041819D
:106160009727000093870703AA97882341473305A1
:10617000A7408280B3C7A5008D8B3307C50081E798
:106180008D4763EDC700AA87637EE50894218507E4
:106190008505A38FD7FEE3EBE7FE8280937635007B
:1061A000AA8789CA942185078505A38FD7FE93F610
:1061B0003700C5BF9376C7FF138606FE63F0C70698
:1061C00083A3050083A2450083AF850003AFC5000C
:1061D00083AE050103AE450103A3850183A8C50174
:1061E0009385450223A0770003A8C5FF23A257008B
:1061F00023A4F70123A6E70123A8D70123AAC701F7
:1062000023AC670023AE17019387470223AE07FF35
:1062100075B790419107910523AEC7FEE3EBD7FE1A
:10622000E3E6E7F6828039713EDA2ED232D436D6F2
:106230003AD842DC46DE9387818122CC804326CA4D
:1062400006CEAA8409C41C4C99E3228505250C447A
:1062500054102686228536C6EF00905BF2406244D9
:10626000D24421618280011126CA4AC806CE22CCBE
:106270004EC652C4AA842E8901C51C4D91E3FD234C
:106280009C4C804499E32685D5239727000093876B
:106290006702631BF402C0405E24A18BB1C71C4897
:1062A000A1C7FD59294A1C4483450900FD17B1E9DE
:1062B0001CC463DD07062286A94526857522FD5785
:1062C0006308F502294535A09727000093878700CA
:1062D0006314F4008044C9B797270000938787FBB5
:1062E000E31CF4FAC0444DBFA2852685252C55D960
:1062F0007D55F2406244D2444249B249224A056186
:1063000082801CC4050963D70700184C63CAE700E4
:10631000638845011C401387170018C08CA361B720
:10632000228626859122E31035F9D9B71C401387C0
:10633000170018C0294798A371B793878181AA8550
:1063400088436FF05FF241119387818122C48043BB
:1063500026C206C61C5CAA8495EB6145EF00007757
:10636000B737CDAB08DC9387E7301CC1B7176DE6B4
:10637000938747235CC1B7E705009387C7EE1CC529
:10638000AD475EA50547814718C95CC91C5CB24092
:10639000224484CB23AA0700924441018280411108
:1063A0009387818122C4804306C61C5C8DEB6145C6
:1063B000312FB737CDAB08DC9387E7301CC1B71757
:1063C0006DE6938747235CC1B7E705009387C7EE67
:1063D0001CC5AD475EA50547814718C95CC9105C5F
:1063E0003787954CB7F75158144A484A1307D7F2E4
:1063F0009387D742B387F602B24022443305E502C1
:106400003E95B387E60233B7E6029386170014CAB7
:106410002A9733B5F6003A9548CA06050581410129
:10642000828035713ECBB707008093C7F7FF3ECE21
:106430003EC8C1779387872032C536C73AC942CD57
:1064400046CF3ECA938781812AC42ACC884334012F
:106450002E862C0086DE36C2EF00500EA247238027
:106460000700F6500D618280011122CC26CA4AC86D
:1064700006CE4EC6AA842E89328401C51C4D91E3F6
:10648000F526972700009387E7E26317F406C040DC
:106490001C4C1CC45E24A18BC1C31C48B5CF1C4836
:1064A00008409379F90F1379F90F1D8D5C48634605
:1064B000F500A2852685692C25E51C440505FD17F8
:1064C0001CC41C401387170018C0238037015C4888
:1064D0006388A7005E24858B81CBA9476316F900EA
:1064E000A2852685B5240DEDF24062444A85D2444A
:1064F0004249B2490561828097270000938787DD72
:106500006314F400804469B797270000938787D805
:10651000E310F4F8C044ADBFA2852685212041D107
:106520007D59D9B741119387818126C2844322C402
:106530004AC006C62A892E8489C49C4C99E32685C4
:106540003526972700009387E7D6631BF402C040E7
:106550000317C40093170701C18393F68700ADEAC0
:1065600093F6070195EEA5472320F900136707046A
:106570005AA47D55B240224492440249410182808E
:1065800097270000938707D56314F4008044C9B7A8
:1065900097270000938707D0E31CF4FAC0444DBF4F
:1065A000918B9DC34C5889C9930744046384F500BB
:1065B0004A851523232A04025E242322040093F72C
:1065C000B7FD5EA41C481CC05E2493E787005EA450
:1065D0001C4899EB5E241307002093F70728638576
:1065E000E700A2854A8591295E2413F717001DC391
:1065F0005C4823240400B307F0401CCC1C48014530
:10660000B5FB8317C40013F707082DD793E70704DA
:106610005EA485B7898B014791E3584818C4F9BF38
:10662000DE25011122CC26CA06CE4AC84EC613F773
:106630008700AA842E8479EBD841634DE000B841ED
:10664000634AE0000145F2406244D2444249B24903
:106650000561828058547DD703A9040093963701C1
:1066600023A0040063DB060670485E24918B99C763
:106670005C401D8E5C5899C33C401D8E5C540C5090
:10668000814626858297FD575A24631DF500944064
:10669000F54763E8D706B70740208507B3D7D7008B
:1066A000858BA5C31C48232204001CC09317370107
:1066B00063D80700FD576314F5009C4091E368C858
:1066C0004C5823A02401BDDD930744046384F500E6
:1066D00026851121232A0402B5B70C5001468546B0
:1066E00026850297FD572A86E311F5F89C40B5DF11
:1066F00075476385E70059476393E70423A02401A6
:1067000091B7136707045AA47D5535BF83A90501C6
:10671000E38A09F203A905008D8B23A03501330913
:106720003941014791E3D84918C4E35D20F11C5475
:106730000C50CA864E86268582976347A0005E2449
:1067400093E707045EA4C9B7AA993309A940F1BF2A
:106750009C49A5C3011122CC06CE2A8411C51C4D2B
:1067600081E72EC62122B24597270000938787B480
:10677000639CF5004C408397C5009DC72285624409
:10678000F24005616FF0DFE997270000938787B437
:106790006394F5000C44C5B797270000938787AF33
:1067A000E39BF5FC4C44C1BFF240624401450561E6
:1067B000828001458280411122C406C62A844EA5EA
:1067C00072A523200500232205002324050023228F
:1067D000050623280500232A0500232C0500214651
:1067E00081451305C505EF90BF9B97170000938760
:1067F00067E85CD097170000938787EA1CD4971747
:106800000000938767EE5CD4971700009387C7F06A
:1068100000D01CD8B240224441018280970500007C
:10682000938545F391AA411126C2130680069384ED
:10683000F5FFB384C4024AC02E8922C406C69385DC
:106840004407352E2A8401CD23200500232225016B
:10685000310508C4138684068145EF907F94228514
:10686000B240224492440249410182801C4DA5E776
:10687000411106C622C497070000938767FA1CD50A
:106880009387C1819C4323240504232605042328E0
:1068900005046314F50085471CCD2A84352848C0BB
:1068A00022851D2808C42285052848C44840014681
:1068B0009145EFF05FF008440546A545EFF0BFEFC6
:1068C00048440946C945EFF01FEF85471CCCB2404C
:1068D000224441018280828041119387C18126C276
:1068E00084434AC006C69C4C22C42A8981E7268577
:1068F000EFF0DFF7938484048044DC40FD1763D617
:1069000007009C40B9CF8440C5BF0317C40039E7D6
:10691000C1778507232204062320040023220400D4
:10692000232404005CC423280400232A0400232C0D
:106930000400214681451305C405EF907F86232A74
:106940000402232C040223240404232604042285A5
:10695000B2402244924402494101828013048406D9
:1069600071BF91454A85EFF01FEC88C049FDB147E2
:106970002320F9000144E1BF797122D44AD052CCDE
:1069800056CA5AC85EC606D626D24ECE2A8AAE8AC5
:10699000130485040149054BFD5B09ECB2502254F8
:1069A0004A8592540259F249624AD24A424BB24B4A
:1069B00045618280044483294400FD1963D40900A1
:1069C0000040E1BFDE24637BFB008397E400638724
:1069D0007701A6855285829A3369A900938484063B
:1069E000E9BF1971A6DAAE848395E500A2DC86DEE4
:1069F000328463DB0500DE2423A0060093F707083A
:106A000085E7930700401DA0300836C6EF005056BA
:106A1000B246E34205FE7247BD67F98F7977BA97B0
:106A200093B717009CC2F1BF930700041CC0F65037
:106A30006654D654014509618280DE25011122CCBD
:106A400006CE26CA4AC8898B2E8489CF9307740440
:106A50001CC01CC885475CC8F2406244D24442490D
:106A60000561828074003000AA84EFF09FF7A24590
:106A70002A892685292219E98317C40013F70720DC
:106A800061FFF19B93E727005EA4C9B79707000059
:106A9000938707D99CD45E2408C008C893E70708E9
:106AA0005EA4A2475CC8B24781CF8315E400268567
:106AB000EF00B04E11C55E24F19B93E717005EA472
:106AC0005E243369F9002316240179B79387818105
:106AD000AA8588436DA0DDC183A7C5FF411122C4EB
:106AE00006C626C21384C5FF63D307003E94AA845A
:106AF000EF00D055938741899C4381EF2322040006
:106B000023AA81882244B2402685924441016F0025
:106B10001054637EF40014403307D4006396E700FA
:106B20009843DC43369718C05CC0D9BFBA87D843B6
:106B300019C3E37DE4FE94433386D700631F8600C8
:106B40001040B29694C33386D700E31DC7FA1043B2
:106B50005843B29694C3D8C375B76375C400B147A0
:106B60009CC04DB71040B306C4006316D700144351
:106B70005843B29614C058C0C0C369B7828001118F
:106B800026CA93843500F19806CE22CC4AC84EC658
:106B9000A104B14763F5F404B14463E4B4042A8961
:106BA000EF00D04A9387418998433A8429E4938738
:106BB00081899C4399E781454A85EF00D02823AC21
:106BC000A188A6854A85EF001028FD59631935076D
:106BD000B1472320F9004A85EF00704729A0E3DE82
:106BE00004FAB1471CC10145F2406244D244424913
:106BF000B249056182801C40858F63CF0702AD4694
:106C000063F6F6001CC03E9404C031A05C406313E0
:106C1000870223AAF1884A85EF0070431305B40068
:106C20009307440061993307F5405DDF3A94898FFB
:106C30001CC05DBF5CC3C5B72287404085BF13043D
:106C400035007198E30285FCB305A4404A85EF0046
:106C5000901FE31B35FBADBF01114AC803A9850096
:106C600022CC52C45AC006CE26CA4EC656C22E8464
:106C7000328B368A63E92609DE2513F7074851C3AC
:106C800004408C495848AA8AB389B4408D44B384DF
:106C9000E4020947B3C4E402138716004E9763F376
:106CA000E400BA8493F70740BDCFA6855685EFF080
:106CB0001FED2A891DE1B14723A0FA005E247D550E
:106CC00093E707045EA4F2406244D2444249B249C9
:106CD000224A924A024B056182800C484E86EFF0B0
:106CE0006FC95E2493F7F7B793E707085EA42328DC
:106CF000240144C84E99B38434412320240104C4A0
:106D0000528963732A01528908404A86DA85EF0066
:106D1000902F1C440145B38727411CC41C403E9959
:106D2000232024014DB726865685EF0070322A892C
:106D30005DFD0C485685EFF01FDAB5BFDE25717199
:106D400026D34AD14ECF06D722D552CD56CB5AC9DB
:106D50005EC762C566C393F70708AA892E89B28405
:106D6000B9C39C49A9E39305000436C6EFF03FE19F
:106D70002320A9002328A900B24615E1B14723A08A
:106D8000F9007D55BA502A549A540A59FA496A4A68
:106D9000DA4A4A4BBA4B2A4C9A4C4D61828093078F
:106DA0000004232AF90093070002A30CF1029307C1
:106DB000000302DA230DF10236CE930B5002971A2C
:106DC0000000938A2A53054C294B26841C2099C322
:106DD00063997709B30C9440638E0C00E68626868F
:106DE000CA854E85EFF05FE7FD57630BF518D25665
:106DF000E69636DA1C2063850718FD5793041400C5
:106E000002D002D63ED202D4A301010682DC8C203D
:106E100015465685EF00B01D13841400825721E5F6
:106E200013F7070109C713070002A301E10613F7CF
:106E3000870009C71307B002A301E10694201307D6
:106E4000A002638AE602B2572684814625461820AE
:106E500093051400130707FD6372E6068DC63ED640
:106E60001DA00504A5B7330555413315AC00C98FE6
:106E70003ED0A28469BF724793064700184336CEBE
:106E8000634707023AD618209307E002631DF70410
:106E900018309307A002631BF702F2470904138717
:106EA00047009C433ACE63C107023ED22DA8330768
:106EB000E04093E727003AD63ED0F1B7B3876703A7
:106EC00085462E84BA9761B7FD57C5B7050402D22F
:106ED000814681472546182093051400130707FDB6
:106EE0006376E606F9F20C200D461715000013052F
:106EF000E540EF00D00F11CD9717000093870740B2
:106F00001D8D93070004B397A700025505045D8DFE
:106F10002AD00C201946171500001305653E93046E
:106F20001400230CB102EF00900C25C59797FFFFCA
:106F30009387470D95E70257F2471377071009CF5C
:106F400091073ECED257D2973EDA41B5B387670359
:106F500085462E84BA9741B79D07E19BA107D5B717
:106F6000780897060000938666CF4A860C104E85F7
:106F700097000000E7000000FD572A8AE314F5FCA3
:106F80008357C9007D5593F70704E39D07DE5255EB
:106F9000D5BB780897060000938646CC4A860C102D
:106FA0004E850921D1BF1C46FD171CC663DA0700B8
:106FB000184E63C5E700A9476394F5006FF0CFCA88
:106FC0001C422E851387170018C28CA382800111E2
:106FD00022CC26CA4AC84EC652C406CE2A89AE89D9
:106FE0003284B304D6007D5A63149400014509A885
:106FF0000C204E864A85EFF01FFB0504E31645FF83
:10700000F2406244D2444249B249224A0561828038
:10701000357122CD26CB4AC94EC706CF52C556C3BD
:107020005AC1DEDEE2DCE6DAAA89AE843289368431
:1070300009C51C4D99E3EFF07F83971700009387F4
:1070400067276398F40C83A44900DE24A18BE5C76D
:107050009C48F5C393070002A304F10293070003C1
:1070600002D22305F10222C6930B5002971A0000A8
:10707000938A4A28054C294B4A841C2099C3639F54
:10708000770DB30C2441638E0C00E6864A86A685F4
:107090004E85EFF0DFF3FD57630FF51C9256E69631
:1070A00036D21C206389071CFD571309140002C83F
:1070B00002CE3ECA02CCA309010482D48345090052
:1070C000154656852D2713041900C24751E913F7B9
:1070D000070109C713070002A309E10413F787009A
:1070E00009C71307B002A309E10483460900130787
:1070F000A002638FE606F2474A848146254618209F
:1071000093051400130707FD6377E60AB5CA3ECE60
:1071100085A8971700009387E71B6395F40083A465
:10712000890025B7971700009387C716E39FF4F0EF
:1071300083A4C90019BFA6854E85EFF0AFBE19D94B
:107140007D55FA406A44DA444A49BA492A4A9A4A79
:107150000A4BF65B665CD65C0D618280050431BF2C
:10716000330555413315AC00C98F3EC82289B9B7E4
:10717000324793064700184336C6634707023ACEA4
:1071800018209307E002631DF70418309307A0024C
:10719000631BF702B2470904138747009C433AC6B2
:1071A00063C107023ECA2DA83307E04093E72700DA
:1071B0003ACE3EC8F1B7B387670385462E84BA97A7
:1071C0003DBFFD57C5B7050402CA81468147254624
:1071D000182093051400130707FD6374E606F9F2FF
:1071E0000C200D461715000013054511092511CD7A
:1071F00097170000938787101D8D93070004B3979E
:10720000A700424505045D8D2AC80C2019461715B4
:1072100000001305E50E130914002304B102C12B6D
:1072200035C19797FFFF9387E7DD95E74247B24760
:107230001377071009CF91073EC69257D2973ED2D7
:1072400025BDB387670385462E84BA9751B79D073E
:10725000E19BA107D5B7780097060000938666D713
:1072600026860C084E8597000000E7000000FD57B9
:107270002A8AE314F5FCDE2493F70704E39207EC73
:107280001255C1B5780097060000938686D42686ED
:107290000C084E85012AE1BF797156CA9C49BA8A09
:1072A000984522D426D24ECE52CC06D64AD05AC8C1
:1072B0005EC6AA892E84B284368A63D3E700BA8771
:1072C0009CC00347340419C385079CC01C4093F736
:1072D000070281C79C4089079CC0032904001379D9
:1072E0006900631A0900130B9401FD5B5C4498402C
:1072F000998F634CF9041C408346340493F70702CA
:10730000B336D000A5EB13063404D2854E85829A9D
:10731000FD576303F5041C4011469840998B544473
:1073200081446397C700B384E64063D3040081447B
:107330001C4418486354F700998FBE9401496904AE
:107340007D5B63982405014509A885465A86D28548
:107350004E85829A631E75017D55B2502254925417
:107360000259F249624AD24A424BB24B456182808D
:107370000509ADBF3307D40013060003A301C704FA
:107380000347540493871600A2978906A381E70454
:107390009DBF85462286D2854E85829AE30E65FB87
:1073A000050945B7797122D426D24AD04ECE06D6E9
:1073B00052CC56CA5AC8B689942D93079006328982
:1073C000AA842E8413863504638DF60263E2D70601
:1073D000930780056386F61863EDD700638E062059
:1073E00093073004638EF60A930A24042301D4041D
:1073F000C9A0930730066385F60A93074006E39514
:10740000F6FE1C40084393F6070893054500C5C6E1
:107410001C410CC363D807001307D002B307F04028
:10742000A301E40497160000938606EE294765A899
:10743000930700076382F61663E5D7029307E00619
:107440006389F6189307F006E390F6FA0C401C43A4
:1074500013F80508138547006307080608C39C4313
:1074600085A893075007E383F6FE93078007638997
:10747000F61293073007E399F6F61C43D041814595
:107480009386470014C383AA070056858D2601C53D
:107490003305554148C05C401CC8A301040461A8E1
:1074A0001C43930A2404938647009C4314C323017E
:1074B000F4048547D5B793F607041C410CC3B9DA29
:1074C000C207C18781BF93F5050408C3C9D99E23AC
:1074D0001307F0066387E60E971600009386C6E250
:1074E0002947A30104044C400CC463C505000840AF
:1074F0006D9908C099E3B28A89CDB28AB3F5E702E3
:10750000FD1AB6958C212380BA00B3D5E70263F04B
:10751000E70CA147631EF7001C40858B91CB5840B8
:107520001C4863C7E70093070003A38FFAFEFD1A08
:107530003306564110C84E87CA867000A28526853C
:10754000EFF09FD57D5A631D450B7D55B2502254F7
:1075500092540259F249624AD24A424B45618280B2
:10756000A382D50497160000938606DA0C400843E0
:1075700013F805081C411105630D080208C313F731
:10758000150001C793E505020CC04147B9FB0C404B
:1075900093F5F5FD0CC0B1B79C4193E707029CC180
:1075A00093078007A302F40497160000938606D77A
:1075B00075BF13F8050408C3E30308FCC207C183C1
:1075C0007DBF97160000938626D4214719BFAE874A
:1075D00035B794411C43CC4913F80608138547007E
:1075E0006306080008C39C438CC339A008C393F604
:1075F00006049C43F5DA8EA323280400B28A25BF33
:1076000014485686CA8526858299E30045F51C40B4
:10761000898B8DE7B2474844E35AF5F23E853DB782
:1076200085465686CA8526858299E30065F3050A54
:107630005C443247998FE345FAFEE9BF014A930A59
:1076400094017D5BF5B7411122C42A842E8523AABB
:1076500001B606C6EFA02FE4FD576317F500938728
:1076600041B79C4391C31CC0B24022444101828077
:10767000411122C42E848395E50006C63524634952
:1076800005007C48AA977CC8B24022444101828010
:107690005E247D777D17F98F5EA4FDB7DE2501118D
:1076A00022CC26CA4AC84EC606CE93F70710AA8433
:1076B0002E843289B68991C78395E50089460146B3
:1076C00009225E247D777D17F98F5EA48315E4007F
:1076D0006244F240CE864A86B24942492685D24467
:1076E000056125A8411122C42E848395E50006C6B4
:1076F000C928FD575A24631AF500FD77FD17F98F45
:107700005EA4B2402244410182808567D98F5EA485
:1077100068C8C5BF8395E50005A8411122C42A8425
:107720002E85B285368623AA01B606C6EFA0CFD233
:10773000FD576317F500938741B79C4391C31CC065
:10774000B240224441018280411122C42A842E8504
:1077500023AA01B606C6492AFD576317F500938789
:1077600041B79C4391C31CC0B24022444101828076
:10777000411122C42A842E85B28523AA01B606C6E9
:10778000952AFD576317F500938741B79C4391C332
:107790001CC0B240224441018280411122C42A848B
:1077A0002E8523AA01B606C6A12AFD576317F50048
:1077B000938741B79C4391C31CC0B240224441010E
:1077C0008280411122C42A842E85B285368623AA5E
:1077D00001B606C6252AFD576317F500938741B702
:1077E0009C4391C31CC0B24022444101828093F566
:1077F000F50F2A966314C500014582801C21E38E93
:10780000B7FE0505C5BF63F1A504B386C500637D5A
:10781000D5029345F6FF8147FD176393F5008280FB
:107820003387F600034807003387C7002A972300F1
:107830000701DDB73387F50014233307F50085070B
:1078400014A3E319F6FE82808147E5BF828082801F
:1078500081E5B2856FF0AFB2011122CC06CE26CA07
:107860004AC84EC6328401EEEFF0EFA60149F2405D
:1078700062444A85D2444249B24905618280AE845D
:10788000AA8989282689E37485FEA2854E85EFF0B2
:107890000FAF2A8969DDA6852286EFE0BF8DA68518
:1078A0004E85EFF04FA3E1B7411122C42A842E8503
:1078B000B285368623AA01B606C6B928FD576317D6
:1078C000F500938741B79C4391C31CC0B24022444A
:1078D0004101828083A7C5FF1385C7FF63D50700D9
:1078E000AA959C413E9582809307800523AAF1B614
:1078F0007D5582809307800523AAF1B67D5582804D
:107900009307800523AAF1B601458280930780057D
:1079100023AAF1B67D5582809307800523AAF1B68C
:107920007D55828053797374656D436C6B3A256421
:107930000D0A00004368697049443A253038780DD3
:107940000A00000043616C696272617474696F6E51
:107950005F56616C203A2025640A0000CDCCCC3DF6
:107960006666663F0000F0439A9999999999B93FE4
:10797000CDCCCCCCCCCCEC3F696E2074696D312081
:10798000697271200000000000F07F4500000000D7
:107990000000000000000440000000000000204043
:1079A000000000000000E03F000000000000344044
:1079B00000000000CF4636400000000000002640D6
:1079C0001D130F130213F412E612D712C812B912C4
:1079D000AA129A128A127A126A125912481237128D
:1079E000251213120112EE11DB11C811B511A111EC
:1079F0008D11791164114F113A1125110F11F910E0
:107A0000E310CC10B5109E1087106F1057103F1068
:107A100026100D10F40FDB0FC20FA80F8E0F740F7E
:107A2000590F3F0F240F090FED0ED20EB60E9A0E0E
:107A30007E0E620E460E290E0C0EF00DD30DB60D05
:107A4000980D7B0D5E0D400D220D050DE70CC90C48
:107A5000AB0C8D0C6F0C510C330C150CF70BD90BB8
:107A6000BB0B9C0B7E0B600B420B240B060BE80A36
:107A7000CA0AAD0A8F0A710A540A360A190AFC09A1
:107A8000DF09C209A50988096C094F0933091709DB
:107A9000FB08DF08C308A8088D08720857083C08CF
:107AA00021080708ED07D307B907A00786076D0768
:107AB00054073C0723070B07F306DB06C406AD0695
:107AC00096067F06680652063C0626061006FB054B
:107AD000E605D105BC05A70593057F056B0558058F
:107AE000450532051F050C05FA04E804D604C40454
:107AF000B304A10490047F046F045F044E043E04A9
:107B00002F041F0410040104F203E303D503C70389
:107B1000B903AB039D0390038203750368035C0301
:107B20004F03430336032A031F0313030703FC0217
:107B3000F102E602DB02D102C602BC02B202A702D7
:107B40009E0294028A02810277026E0265025C0242
:107B500054024B0242023A0232022A0222021A0262
:107B600012020B020302FC01F401ED01E601DF0148
:107B7000D801D201CB01C401BE01B801B101AB01F2
:107B8000A5019F01990194018E01880183017D0166
:107B9000780173016E01690163015E015A015501AB
:107BA0005001000000401C460000C8420000904107
:107BB000547269636B6C6500666C6F6174000000E1
:107BC00000008041000000419A9999999999A93F34
:107BD0009A9999999999C93F17B75138ACC52737E0
:107BE0006F12033ABD37863500007A440AD7A33BAB
:107BF0000000003FC853023E5B494E464F5D205B8C
:107C000025733A25645D20526567697374726174E7
:107C1000696F6E2073756363657373200D0A0D0AB7
:107C2000000000005B4552524F525D205B25733AC5
:107C300025645D202052656769737465725F4E75B7
:107C40006D626572206572726F723A2578200D0A36
:107C50000D0A00005B4552524F525D205B25733A7E
:107C600025645D202052656769737465725F537483
:107C70006172745F41646472657373206572726FC0
:107C800072203A202578200D0A0D0A00696E2077AF
:107C9000726974652072656769737465722000008B
:107CA0005B494E464F5D205B25733A25645D20207D
:107CB000534C5F52656164526567697374657242C3
:107CC000617474657279566F6C74616765200D0A12
:107CD000000000005B494E464F5D205B25733A254E
:107CE000645D2020534C5F5265616452656769731F
:107CF000746572436861726743757272656E742051
:107D00000D0A00005B494E464F5D205B25733A2506
:107D1000645D2020534C5F526561645265676973EE
:107D200074657244697363686172674375727265E2
:107D30006E74200D0A0000005B494E464F5D205BCB
:107D400025733A25645D2020534C5F52656164526F
:107D50006567697374657244697363686172674DBE
:107D60006F735374617465200D0A00000000204198
:107D70005B494E464F5D205B25733A25645D2020AC
:107D8000534C5F52656164526567697374657248EC
:107D9000696768536964654D6F7354656D7065728A
:107DA0006174757265200D0A000000005B494E4643
:107DB0004F5D205B25733A25645D2020534C5F5254
:107DC00065616452656769737465724D5050544DB6
:107DD0006F6465200D0A00005B494E464F5D205BD5
:107DE00025733A25645D2020534C5F5265616452CF
:107DF00065676973746572536F6C61724F70656EFD
:107E000043697263756974566F6C74616765200DA0
:107E10000A0000005B494E464F5D205B25733A2502
:107E2000645D204D617463685F5374617274666C45
:107E300061672073756363657373200D0A0D0A0013
:107E40005B494E464F5D205B25733A25645D204DAE
:107E5000617463685F6164647265737320737563D2
:107E600063657373200D0A0D0A0000005B494E46DE
:107E70004F5D205B25733A25645D204D6174636816
:107E80005F42726F6164636173746164647265738D
:107E90007320737563636573730D0A0D0A00000028
:107EA0005B494E464F5D205B25733A25645D205249
:107EB0006561645F52656769737465720D0A0D0AC6
:107EC000000000005B494E464F5D205B25733A255C
:107ED000645D2057726974655F5265676973746584
:107EE000720D0A0D0A0000005B494E464F5D205B93
:107EF00025733A25645D204F74686572206672614F
:107F00006D65730D0A0D0A005B494E464F5D205B9F
:107F100025733A25645D2042726F616463617374F6
:107F20005F5363616E0D0A0D0A0000005B494E4607
:107F30004F5D205B25733A25645D20526567697348
:107F400074726174696F6E5F726571756573740DBB
:107F50000A0D0A005B494E464F5D205B25733A25AA
:107F6000645D2066756E636F6465206572726F7202
:107F70002025780D0A0D0A0020647574795F7261FE
:107F800074696F203A2025642F31303030200A0088
:107F900020766F7574203A2025642F313030200A06
:107FA00000000000207642617474657279203A20E6
:107FB00025642F313030200A0000000020496F7501
:107FC00074203A2025642F313030200A0000000050
:107FD00020496469736F7574203A2025642F31300D
:107FE00030200A00206D6F7354203A2025642F3111
:107FF00030200A00206D6F735374617465203A203D
:108000002564200A0000000020302EC3BBD3D0B965
:10801000A4D7F73B20312EE4B8C1F7C4A3CABD3BB7
:1080200020322EBAE3C1F7C4A3CABD3B20332EBA17
:10803000E3D1B9C4A3CABD3B20342EB8A1B3E4C474
:10804000A3CABD3B20352EC3BBD3D0B5E7B3D820E0
:108050003A202564200A00007B14AE47E17A843F71
:10806000766F6C7420696E203A2025642F31303091
:10807000200A00000000803F000010412068656C6D
:108080006C6F20776F726C64200A00003333333FCB
:1080900072C4FFFF64C3FFFF64C3FFFF62C3FFFF3F
:1080A0006AC3FFFF6AC3FFFF30C3FFFF62C3FFFF66
:1080B0006AC3FFFF30C3FFFF6AC3FFFF62C3FFFF56
:1080C0005EC4FFFF5EC4FFFF5EC4FFFF30C3FFFF5F
:1080D000AED3FFFFD4D2FFFFA8D3FFFFDCD2FFFF58
:1080E000A8D3FFFFA2D2FFFFA8D3FFFFDCD2FFFF80
:1080F000D4D2FFFFD4D2FFFFA2D2FFFFDCD2FFFF1A
:10810000E2D2FFFFE2D2FFFFE2D2FFFFA2D2FFFFE7
:1081100094D2FFFF94D2FFFF68D3FFFF44D4FFFF48
:1081200068D3FFFF62D2FFFF68D3FFFF44D4FFFF95
:1081300094D2FFFF94D2FFFF62D2FFFF44D4FFFF2F
:10814000A2D2FFFFA2D2FFFFA2D2FFFF62D2FFFFA7
:10815000BCD6FFFF0AD6FFFF0AD6FFFF08D6FFFFF7
:108160000ED6FFFF0ED6FFFFDED5FFFF08D6FFFFBE
:108170000ED6FFFFDED5FFFF0ED6FFFF08D6FFFFAE
:10818000AAD6FFFFAAD6FFFFAAD6FFFFDED5FFFFC4
:1081900000010202030303030404040404040404AE
:1081A000050505050505050505050505050505057F
:1081B000060606060606060606060606060606065F
:1081C000060606060606060606060606060606064F
:1081D000070707070707070707070707070707072F
:1081E000070707070707070707070707070707071F
:1081F000070707070707070707070707070707070F
:1082000007070707070707070707070707070707FE
:1082100008080808080808080808080808080808DE
:1082200008080808080808080808080808080808CE
:1082300008080808080808080808080808080808BE
:1082400008080808080808080808080808080808AE
:10825000080808080808080808080808080808089E
:10826000080808080808080808080808080808088E
:10827000080808080808080808080808080808087E
:10828000080808080808080808080808080808086E
:1082900000000000000000000000000000000000DE
:1082A00000000000000000000000000000000000CE
:1082B00000000000000000000000000000000000BE
:1082C00000000000000000000000000000000000AE
:1082D000000000000000000000000000000000009E
:1082E000000000000000000000000000000000008E
:1082F000232D302B20000000686C4C00656667451C
:108300004647000030313233343536373839414250
:1083100043444546000000003031323334353637AF
:0C8320003839616263646566000000008B
:10832C000000000000000000010203040607080919
:10833C0000000000010203040102030406070809FF
:10834C0000000000000000000000000000E80378BE
:10835C00050500A406DC05A005640003000A000165
:10836C00000100140046003200280000534C11118B
:10837C001111111111010001001600003000000054
:10838C00D2290000100000005C270000A0000000B3
:10839C0028270000A1000000D8260000D000000013
:1083AC0034290000D10000009628000001010000D3
:1083BC009C26000002010000602600000301000062
:1083CC002426000004010000E62500000501000041
:1083DC00A82500000601000084250000070100000C
:1083EC005A2500000000000003000000802500005A
:1083FC000000000000000000000000000000000071
:10840C0000000000040000008025000000000000B7
:10841C000000000000000000000000000000000050
:10842C00B0820000D08200009082000000000000AA
:10843C000000000000000000000000000000000030
:10844C000000000000000000000000000000000020
:10845C000000000000000000000000000000000010
:10846C000000000000000000000000000000000000
:10847C0000000000000000000000000000000000F0
:10848C00006CDC0202040608D8040020CDCC4C3F62
:10849C000101010101010000FC000020FC00002092
:00000001FF
